:10000000FCC1000020C200001EC200001CC2000093
:100010001AC2000018C2000016C2000014C200007C
:1000200012C2000010C200000EC200000CC200008C
:100030000AC200000C94590E4AC4000080C400009B
:100040000C949E2EB4C40000EAC4000020C5000039
:1000500056C500008CC50000C2C50000F8C50000F0
:10006000F2C100000C94EB2FEEC10000ECC10000C7
:100070000C946D15E8C10000E6C10000E4C1000069
:10008000E2C10000E0C10000DEC10000DCC10000F0
:10009000DAC10000D8C10000D6C1000014C30000BE
:1000A0004FC300008AC30000C5C30000CCC10000DC
:1000B000CAC10000C8C100000C94BD0E0C948F088A
:1000C0000C94C7080C94FF080C9437090C946F0922
:1000D0000C94A7090C94DF090C94170A0C944F0A8E
:1000E0000C94870AB0C10000AEC10000ACC1000092
:1000F000AAC10000A8C10000A6C10000A4C1000060
:100100000C9496170C94CE140C94291D9CC10000DD
:100110009AC1000098C1000096C10000E0C1000033
:100120001BC2000056C2000091C200008CC100003A
:100130000C948B0EC4C50000FAC5000030C6000048
:1001400066C600009CC60000D2C6000008C70000BA
:100150003EC7000074C70000AAC7000074C10000B9
:1001600072C1000070C100006EC100006CC10000CF
:100170006AC1000068C1000066C1000064C10000DF
:1001800062C1000060C100005EC100005CC10000EF
:100190005AC1000058C1000056C1000054C10000FF
:1001A00052C1000050C100004EC100000C94EF0E7F
:1001B0000C94BF0A0C94F70A0C942F0B0C94670B49
:1001C0000C949F0B0C94D70B0C940F0C0C94470CB5
:1001D0000C947F0C0C94B70C36C1000034C10000A5
:1001E00032C1000030C100002EC100002CC100004F
:1001F0002AC1000028C1000026C10000FA120D1318
:1002000020133313461359136C137F13036EDB361D
:100210003D9A9999993DABAAAA2A3E000000803FD9
:10022000084AD73B3BCE016E84BCBFFDC12F3D6C5D
:1002300074319ABD56833DDA3D00C77F11BED9E4C3
:10024000BB4C3E916BAAAABE000000803F072C7AEF
:10025000A5BA6CC590DA3B9365FC8BBC53F810FDD6
:100260003C5692834DBD879D3AB63DCBC9BF5BBE20
:1002700073DA0FC93F08000000BE922449123EAB5A
:10028000AAAA2ABECDCCCC4C3E00000080BEABAAB0
:10029000AAAA3E00000000BF000000803F0000004E
:1002A0000000084178D3BB4387D1133D190E3CC3EE
:1002B000BD4282AD2B3E68EC8276BED98FE1A93E6D
:1002C0004C80EFFFBE01C4FF7F3F0000000000072D
:1002D000634236B79BD8A71A39685618AEBAAB55E1
:1002E0008C1D3CB7CC5763BD6DEDFD753EF61772A6
:1002F00031BF000000803F006E616E00696E6600D5
:1003000000407A10F35A00A0724E18090010A5D4CC
:10031000E80000E87648170000E40B54020000CA29
:100320009A3B000000E1F50500008096980000006F
:1003300040420F000000A0860100000010270000CE
:100340000000E803000000006400000000000A0054
:10035000000000000100000000002C76D888DC6757
:100360004F0823DFC1DFAE59E1B1B796E5E3E453AF
:10037000C63AE651997696E8E6C28426EB898C9BCC
:1003800062ED407C6FFCEFBC9C9F40F2BAA56FA56C
:10039000F490055A2AF75C936B6CF9676DC11BFCEE
:1003A000E0E40D47FEF520E6B500D0ED902E030009
:1003B000943577050080841E080000204E0A000056
:1003C00000C80C333333330F986E12831141EF8D15
:1003D0002114893BE65516CFFEE6DB18D1844B3855
:1003E0001BF77C1D901DA4BBE424203284725E2286
:1003F0008100C9F124ECA1E53D2711241FBECFEFF8
:10040000CDBFDFE3DEBF00E00CBF18BE19BE1ABED1
:100410001BBE11E2A0E0B0E2EEE3F8E700E00BBFA4
:1004200002C007900D92A23CB107D9F71BBE29E28A
:10043000A2ECB1E201C01D92AD3AB207E1F70E9411
:10044000CE300C941D3CDCCDCF93DF931F921F92D6
:10045000CDB7DEB78FEF80937000809371008093EB
:100460007200809373008093740080937500809372
:1004700076008FB78A83F8949A81E0E5F0E0808176
:10048000826080839FBF818181FFFDCF61E080E436
:1004900090E00DD28FB78983F8949981E0E5F0E080
:1004A00080818E7F80839FBF0F900F90DF91CF91CF
:1004B0000895CF93DF931F92CDB7DEB79FB799838F
:1004C000F8949981E82FF0E0E059FF4F6095808122
:1004D000682360839FBF0F90DF91CF9108951F9293
:1004E0000F920FB60F92112408B60F9218BE09B6DC
:1004F0000F9219BE0BB60F921BBE2F933F934F93D3
:100500005F936F937F938F939F93AF93BF93EF937B
:10051000FF934091240250912502E0913925F091FA
:100520003A2561E080E092E01995FF91EF91BF914B
:10053000AF919F918F917F916F915F914F913F917B
:100540002F910F900BBE0F9009BE0F9008BE0F9019
:100550000FBE0F901F9018951F920F920FB60F921B
:10056000112408B60F9218BE09B60F9219BE0BB629
:100570000F921BBE2F933F934F935F936F937F9385
:100580008F939F93AF93BF93EF93FF9340912C0270
:1005900050912D02E0913925F0913A2562E080E0FA
:1005A00092E01995FF91EF91BF91AF919F918F913B
:1005B0007F916F915F914F913F912F910F900BBE63
:1005C0000F9009BE0F9008BE0F900FBE0F901F90A6
:1005D00018951F920F920FB60F92112408B60F9222
:1005E00018BE09B60F9219BE0BB60F921BBE2F9301
:1005F0003F934F935F936F937F938F939F93AF93AB
:10060000BF93EF93FF934091340250913502E091F4
:100610003925F0913A2564E080E092E01995FF9148
:10062000EF91BF91AF919F918F917F916F915F916A
:100630004F913F912F910F900BBE0F9009BE0F90DD
:1006400008BE0F900FBE0F901F9018951F920F922B
:100650000FB60F92112408B60F9218BE09B60F926A
:1006600019BE0BB60F921BBE2F933F934F935F9310
:100670006F937F938F939F93AF93BF93EF93FF936A
:1006800040913C0250913D02E0913925F0913A258C
:1006900068E080E092E01995FF91EF91BF91AF91F2
:1006A0009F918F917F916F915F914F913F912F918A
:1006B0000F900BBE0F9009BE0F9008BE0F900FBE9B
:1006C0000F901F9018951F920F920FB60F92112442
:1006D00008B60F9218BE09B60F9219BE0BB60F924C
:1006E0001BBE2F933F934F935F936F937F938F9393
:1006F0009F93AF93BF93EF93FF9340916402509108
:100700006502E0913725F091382561E080E492E0C0
:100710001995FF91EF91BF91AF919F918F917F912B
:100720006F915F914F913F912F910F900BBE0F9062
:1007300009BE0F9008BE0F900FBE0F901F90189526
:100740001F920F920FB60F92112408B60F9218BE87
:1007500009B60F9219BE0BB60F921BBE2F933F9393
:100760004F935F936F937F938F939F93AF93BF93B9
:10077000EF93FF9340916C0250916D02E091372509
:10078000F091382562E080E492E01995FF91EF91B5
:10079000BF91AF919F918F917F916F915F914F9199
:1007A0003F912F910F900BBE0F9009BE0F9008BE86
:1007B0000F900FBE0F901F9018951F920F920FB6BB
:1007C0000F92112408B60F9218BE09B60F9219BEE7
:1007D0000BB60F921BBE2F933F934F935F936F9374
:1007E0007F938F939F93AF93BF93EF93FF9340912A
:1007F000740250917502E0913725F091382564E03C
:1008000080E492E01995FF91EF91BF91AF919F9194
:100810008F917F916F915F914F913F912F910F90A9
:100820000BBE0F9009BE0F9008BE0F900FBE0F9029
:100830001F9018951F920F920FB60F92112408B6B1
:100840000F9218BE09B60F9219BE0BB60F921BBEBF
:100850002F933F934F935F936F937F938F939F93C8
:10086000AF93BF93EF93FF9340917C0250917D0231
:10087000E0913725F091382568E080E492E0199501
:10088000FF91EF91BF91AF919F918F917F916F9168
:100890005F914F913F912F910F900BBE0F9009BE2A
:1008A0000F9008BE0F900FBE0F901F9018951BBEA3
:1008B000FC0128ED24BF608308954091CA01E62F12
:1008C000F72F8093CA0184914093CA0108951F9223
:1008D0000F920FB60F92112408B60F9218BE09B6E8
:1008E0000F9219BE0BB60F921BBE2F933F934F93DF
:1008F0005F936F937F938F939F93AF93BF93EF9388
:10090000FF93E0910E22F0910F22309709F0199594
:10091000FF91EF91BF91AF919F918F917F916F91D7
:100920005F914F913F912F910F900BBE0F9009BE99
:100930000F9008BE0F900FBE0F901F9018951F923A
:100940000F920FB60F92112408B60F9218BE09B677
:100950000F9219BE0BB60F921BBE2F933F934F936E
:100960005F936F937F938F939F93AF93BF93EF9317
:10097000FF93E0910C22F0910D22309709F0199528
:10098000FF91EF91BF91AF919F918F917F916F9167
:100990005F914F913F912F910F900BBE0F9009BE29
:1009A0000F9008BE0F900FBE0F901F9018951F92CA
:1009B0000F920FB60F92112408B60F9218BE09B607
:1009C0000F9219BE0BB60F921BBE2F933F934F93FE
:1009D0005F936F937F938F939F93AF93BF93EF93A7
:1009E000FF93E0910A22F0910B22309709F01995BC
:1009F000FF91EF91BF91AF919F918F917F916F91F7
:100A00005F914F913F912F910F900BBE0F9009BEB8
:100A10000F9008BE0F900FBE0F901F9018951F9259
:100A20000F920FB60F92112408B60F9218BE09B696
:100A30000F9219BE0BB60F921BBE2F933F934F938D
:100A40005F936F937F938F939F93AF93BF93EF9336
:100A5000FF93E0910822F0910922309709F019954F
:100A6000FF91EF91BF91AF919F918F917F916F9186
:100A70005F914F913F912F910F900BBE0F9009BE48
:100A80000F9008BE0F900FBE0F901F9018951F92E9
:100A90000F920FB60F92112408B60F9218BE09B626
:100AA0000F9219BE0BB60F921BBE2F933F934F931D
:100AB0005F936F937F938F939F93AF93BF93EF93C6
:100AC000FF93E0910622F0910722309709F01995E3
:100AD000FF91EF91BF91AF919F918F917F916F9116
:100AE0005F914F913F912F910F900BBE0F9009BED8
:100AF0000F9008BE0F900FBE0F901F9018951F9279
:100B00000F920FB60F92112408B60F9218BE09B6B5
:100B10000F9219BE0BB60F921BBE2F933F934F93AC
:100B20005F936F937F938F939F93AF93BF93EF9355
:100B3000FF93E0910422F0910522309709F0199576
:100B4000FF91EF91BF91AF919F918F917F916F91A5
:100B50005F914F913F912F910F900BBE0F9009BE67
:100B60000F9008BE0F900FBE0F901F9018951F9208
:100B70000F920FB60F92112408B60F9218BE09B645
:100B80000F9219BE0BB60F921BBE2F933F934F933C
:100B90005F936F937F938F939F93AF93BF93EF93E5
:100BA000FF93E0910222F0910322309709F019950A
:100BB000FF91EF91BF91AF919F918F917F916F9135
:100BC0005F914F913F912F910F900BBE0F9009BEF7
:100BD0000F9008BE0F900FBE0F901F9018951F9298
:100BE0000F920FB60F92112408B60F9218BE09B6D5
:100BF0000F9219BE0BB60F921BBE2F933F934F93CC
:100C00005F936F937F938F939F93AF93BF93EF9374
:100C1000FF93E0910022F0910122309709F019959D
:100C2000FF91EF91BF91AF919F918F917F916F91C4
:100C30005F914F913F912F910F900BBE0F9009BE86
:100C40000F9008BE0F900FBE0F901F9018951F9227
:100C50000F920FB60F92112408B60F9218BE09B664
:100C60000F9219BE0BB60F921BBE2F933F934F935B
:100C70005F936F937F938F939F93AF93BF93EF9304
:100C8000FF93E091FE21F091FF21309709F0199533
:100C9000FF91EF91BF91AF919F918F917F916F9154
:100CA0005F914F913F912F910F900BBE0F9009BE16
:100CB0000F9008BE0F900FBE0F901F9018951F92B7
:100CC0000F920FB60F92112408B60F9218BE09B6F4
:100CD0000F9219BE0BB60F921BBE2F933F934F93EB
:100CE0005F936F937F938F939F93AF93BF93EF9394
:100CF000FF93E091FC21F091FD21309709F01995C7
:100D0000FF91EF91BF91AF919F918F917F916F91E3
:100D10005F914F913F912F910F900BBE0F9009BEA5
:100D20000F9008BE0F900FBE0F901F9018951F9246
:100D30000F920FB60F92112408B60F9218BE09B683
:100D40000F9219BE0BB60F921BBE2F933F934F937A
:100D50005F936F937F938F939F93AF93BF93EF9323
:100D6000FF93E091FA21F091FB21309709F019955A
:100D7000FF91EF91BF91AF919F918F917F916F9173
:100D80005F914F913F912F910F900BBE0F9009BE35
:100D90000F9008BE0F900FBE0F901F9018951F92D6
:100DA0000F920FB60F92112408B60F9218BE09B613
:100DB0000F9219BE0BB60F921BBE2F933F934F930A
:100DC0005F936F937F938F939F93AF93BF93EF93B3
:100DD000FF93E091F821F091F921309709F01995EE
:100DE000FF91EF91BF91AF919F918F917F916F9103
:100DF0005F914F913F912F910F900BBE0F9009BEC5
:100E00000F9008BE0F900FBE0F901F9018951F9265
:100E10000F920FB60F92112408B60F9218BE09B6A2
:100E20000F9219BE0BB60F921BBE2F933F934F9399
:100E30005F936F937F938F939F93AF93BF93EF9342
:100E4000FF93E091F621F091F721309709F0199581
:100E5000FF91EF91BF91AF919F918F917F916F9192
:100E60005F914F913F912F910F900BBE0F9009BE54
:100E70000F9008BE0F900FBE0F901F9018951F92F5
:100E80000F920FB60F92112408B60F9218BE09B632
:100E90000F9219BE0BB60F921BBE2F933F934F9329
:100EA0005F936F937F938F939F93AF93BF93EF93D2
:100EB000FF93E091F421F091F521309709F0199515
:100EC000FF91EF91BF91AF919F918F917F916F9122
:100ED0005F914F913F912F910F900BBE0F9009BEE4
:100EE0000F9008BE0F900FBE0F901F9018951F9285
:100EF0000F920FB60F92112408B60F9218BE09B6C2
:100F00000F9219BE0BB60F921BBE2F933F934F93B8
:100F10005F936F937F938F939F93AF93BF93EF9361
:100F2000FF93E091F221F091F321309709F01995A8
:100F3000FF91EF91BF91AF919F918F917F916F91B1
:100F40005F914F913F912F910F900BBE0F9009BE73
:100F50000F9008BE0F900FBE0F901F9018951F9214
:100F60000F920FB60F92112408B60F9218BE09B651
:100F70000F9219BE0BB60F921BBE2F933F934F9348
:100F80005F936F937F938F939F93AF93BF93EF93F1
:100F9000FF93E091F021F091F121309709F019953C
:100FA000FF91EF91BF91AF919F918F917F916F9141
:100FB0005F914F913F912F910F900BBE0F9009BE03
:100FC0000F9008BE0F900FBE0F901F9018951F92A4
:100FD0000F920FB60F92112408B60F9218BE09B6E1
:100FE0000F9219BE0BB60F921BBE2F933F934F93D8
:100FF0005F936F937F938F939F93AF93BF93EF9381
:10100000FF93E091EE21F091EF21309709F01995CF
:10101000FF91EF91BF91AF919F918F917F916F91D0
:101020005F914F913F912F910F900BBE0F9009BE92
:101030000F9008BE0F900FBE0F901F9018951F9233
:101040000F920FB60F92112408B60F9218BE09B670
:101050000F9219BE0BB60F921BBE2F933F934F9367
:101060005F936F937F938F939F93AF93BF93EF9310
:10107000FF93E091EC21F091ED21309709F0199563
:10108000FF91EF91BF91AF919F918F917F916F9160
:101090005F914F913F912F910F900BBE0F9009BE22
:1010A0000F9008BE0F900FBE0F901F9018951F92C3
:1010B0000F920FB60F92112408B60F9218BE09B600
:1010C0000F9219BE0BB60F921BBE2F933F934F93F7
:1010D0005F936F937F938F939F93AF93BF93EF93A0
:1010E000FF93E091EA21F091EB21309709F01995F7
:1010F000FF91EF91BF91AF919F918F917F916F91F0
:101100005F914F913F912F910F900BBE0F9009BEB1
:101110000F9008BE0F900FBE0F901F9018951F9252
:101120000F920FB60F92112408B60F9218BE09B68F
:101130000F9219BE0BB60F921BBE2F933F934F9386
:101140005F936F937F938F939F93AF93BF93EF932F
:10115000FF93E091E821F091E921309709F019958A
:10116000FF91EF91BF91AF919F918F917F916F917F
:101170005F914F913F912F910F900BBE0F9009BE41
:101180000F9008BE0F900FBE0F901F9018951F92E2
:101190000F920FB60F92112408B60F9218BE09B61F
:1011A0000F9219BE0BB60F921BBE2F933F934F9316
:1011B0005F936F937F938F939F93AF93BF93EF93BF
:1011C000FF93E091E621F091E721309709F019951E
:1011D000FF91EF91BF91AF919F918F917F916F910F
:1011E0005F914F913F912F910F900BBE0F9009BED1
:1011F0000F9008BE0F900FBE0F901F9018951F9272
:101200000F920FB60F92112408B60F9218BE09B6AE
:101210000F9219BE0BB60F921BBE2F933F934F93A5
:101220005F936F937F938F939F93AF93BF93EF934E
:10123000FF93E091E421F091E521309709F01995B1
:10124000FF91EF91BF91AF919F918F917F916F919E
:101250005F914F913F912F910F900BBE0F9009BE60
:101260000F9008BE0F900FBE0F901F9018951F9201
:101270000F920FB60F92112408B60F9218BE09B63E
:101280000F9219BE0BB60F921BBE2F933F934F9335
:101290005F936F937F938F939F93AF93BF93EF93DE
:1012A000FF93E091E221F091E321309709F0199545
:1012B000FF91EF91BF91AF919F918F917F916F912E
:1012C0005F914F913F912F910F900BBE0F9009BEF0
:1012D0000F9008BE0F900FBE0F901F9018951F9291
:1012E0000F920FB60F92112408B60F9218BE09B6CE
:1012F0000F9219BE0BB60F921BBE2F933F934F93C5
:101300005F936F937F938F939F93AF93BF93EF936D
:10131000FF93E091E021F091E121309709F01995D8
:10132000FF91EF91BF91AF919F918F917F916F91BD
:101330005F914F913F912F910F900BBE0F9009BE7F
:101340000F9008BE0F900FBE0F901F9018951F9220
:101350000F920FB60F92112408B60F9218BE09B65D
:101360000F9219BE0BB60F921BBE2F933F934F9354
:101370005F936F937F938F939F93AF93BF93EF93FD
:10138000FF93E091DE21F091DF21309709F019956C
:10139000FF91EF91BF91AF919F918F917F916F914D
:1013A0005F914F913F912F910F900BBE0F9009BE0F
:1013B0000F9008BE0F900FBE0F901F9018951F92B0
:1013C0000F920FB60F92112408B60F9218BE09B6ED
:1013D0000F9219BE0BB60F921BBE2F933F934F93E4
:1013E0005F936F937F938F939F93AF93BF93EF938D
:1013F000FF93E091DC21F091DD21309709F0199500
:10140000FF91EF91BF91AF919F918F917F916F91DC
:101410005F914F913F912F910F900BBE0F9009BE9E
:101420000F9008BE0F900FBE0F901F9018951F923F
:101430000F920FB60F92112408B60F9218BE09B67C
:101440000F9219BE0BB60F921BBE2F933F934F9373
:101450005F936F937F938F939F93AF93BF93EF931C
:10146000FF93E091DA21F091DB21309709F0199593
:10147000FF91EF91BF91AF919F918F917F916F916C
:101480005F914F913F912F910F900BBE0F9009BE2E
:101490000F9008BE0F900FBE0F901F9018951F92CF
:1014A0000F920FB60F92112408B60F9218BE09B60C
:1014B0000F9219BE0BB60F921BBE2F933F934F9303
:1014C0005F936F937F938F939F93AF93BF93EF93AC
:1014D000FF93E091D821F091D921309709F0199527
:1014E000FF91EF91BF91AF919F918F917F916F91FC
:1014F0005F914F913F912F910F900BBE0F9009BEBE
:101500000F9008BE0F900FBE0F901F9018951F925E
:101510000F920FB60F92112408B60F9218BE09B69B
:101520000F9219BE0BB60F921BBE2F933F934F9392
:101530005F936F937F938F939F93AF93BF93EF933B
:10154000FF93E091D621F091D721309709F01995BA
:10155000FF91EF91BF91AF919F918F917F916F918B
:101560005F914F913F912F910F900BBE0F9009BE4D
:101570000F9008BE0F900FBE0F901F9018951F92EE
:101580000F920FB60F92112408B60F9218BE09B62B
:101590000F9219BE0BB60F921BBE2F933F934F9322
:1015A0005F936F937F938F939F93AF93BF93EF93CB
:1015B000FF93E091D421F091D521309709F019954E
:1015C000FF91EF91BF91AF919F918F917F916F911B
:1015D0005F914F913F912F910F900BBE0F9009BEDD
:1015E0000F9008BE0F900FBE0F901F9018951F927E
:1015F0000F920FB60F92112408B60F9218BE09B6BB
:101600000F9219BE0BB60F921BBE2F933F934F93B1
:101610005F936F937F938F939F93AF93BF93EF935A
:10162000FF93E091D221F091D321309709F01995E1
:10163000FF91EF91BF91AF919F918F917F916F91AA
:101640005F914F913F912F910F900BBE0F9009BE6C
:101650000F9008BE0F900FBE0F901F9018951F920D
:101660000F920FB60F92112408B60F9218BE09B64A
:101670000F9219BE0BB60F921BBE2F933F934F9341
:101680005F936F937F938F939F93AF93BF93EF93EA
:10169000FF93E091D021F091D121309709F0199575
:1016A000FF91EF91BF91AF919F918F917F916F913A
:1016B0005F914F913F912F910F900BBE0F9009BEFC
:1016C0000F9008BE0F900FBE0F901F9018951F929D
:1016D0000F920FB60F92112408B60F9218BE09B6DA
:1016E0000F9219BE0BB60F921BBE2F933F934F93D1
:1016F0005F936F937F938F939F93AF93BF93EF937A
:10170000FF93E091CE21F091CF21309709F0199508
:10171000FF91EF91BF91AF919F918F917F916F91C9
:101720005F914F913F912F910F900BBE0F9009BE8B
:101730000F9008BE0F900FBE0F901F9018951F922C
:101740000F920FB60F92112408B60F9218BE09B669
:101750000F9219BE0BB60F921BBE2F933F934F9360
:101760005F936F937F938F939F93AF93BF93EF9309
:10177000FF93E091CC21F091CD21309709F019959C
:10178000FF91EF91BF91AF919F918F917F916F9159
:101790005F914F913F912F910F900BBE0F9009BE1B
:1017A0000F9008BE0F900FBE0F901F9018951F92BC
:1017B0000F920FB60F92112408B60F9218BE09B6F9
:1017C0000F9219BE0BB60F921BBE2F933F934F93F0
:1017D0005F936F937F938F939F93AF93BF93EF9399
:1017E000FF93E091CA21F091CB21309709F0199530
:1017F000FF91EF91BF91AF919F918F917F916F91E9
:101800005F914F913F912F910F900BBE0F9009BEAA
:101810000F9008BE0F900FBE0F901F9018951F924B
:101820000F920FB60F92112408B60F9218BE09B688
:101830000F9219BE0BB60F921BBE2F933F934F937F
:101840005F936F937F938F939F93AF93BF93EF9328
:10185000FF93E091C821F091C921309709F01995C3
:10186000FF91EF91BF91AF919F918F917F916F9178
:101870005F914F913F912F910F900BBE0F9009BE3A
:101880000F9008BE0F900FBE0F901F9018951F92DB
:101890000F920FB60F92112408B60F9218BE09B618
:1018A0000F9219BE0BB60F921BBE2F933F934F930F
:1018B0005F936F937F938F939F93AF93BF93EF93B8
:1018C000FF93E091C621F091C721309709F0199557
:1018D000FF91EF91BF91AF919F918F917F916F9108
:1018E0005F914F913F912F910F900BBE0F9009BECA
:1018F0000F9008BE0F900FBE0F901F9018951F926B
:101900000F920FB60F92112408B60F9218BE09B6A7
:101910000F9219BE0BB60F921BBE2F933F934F939E
:101920005F936F937F938F939F93AF93BF93EF9347
:10193000FF93E091C421F091C521309709F01995EA
:10194000FF91EF91BF91AF919F918F917F916F9197
:101950005F914F913F912F910F900BBE0F9009BE59
:101960000F9008BE0F900FBE0F901F9018951F92FA
:101970000F920FB60F92112408B60F9218BE09B637
:101980000F9219BE0BB60F921BBE2F933F934F932E
:101990005F936F937F938F939F93AF93BF93EF93D7
:1019A000FF93E091C221F091C321309709F019957E
:1019B000FF91EF91BF91AF919F918F917F916F9127
:1019C0005F914F913F912F910F900BBE0F9009BEE9
:1019D0000F9008BE0F900FBE0F901F9018951F9389
:1019E000CF93DF931F921F92CDB7DEB72FB72A8315
:1019F000F8941A81282F392F211588E0380749F4E7
:101A000061E083E00E94590264E083E00E94590291
:101A10005CC0203488E0380749F462E083E00E942B
:101A2000590264E083E00E9459024FC0211589E009
:101A3000380749F461E084E00E94590264E084E0E0
:101A40000E94590242C0203489E0380749F462E01C
:101A500084E00E94590264E084E00E94590235C08B
:101A600021158AE0380749F461E085E00E945902B7
:101A700064E085E00E94590228C020348AE03807DB
:101A800049F462E085E00E94590264E085E00E942A
:101A900059021BC021158BE0380749F461E086E04C
:101AA0000E94590264E086E00E9459020EC0203470
:101AB0003B4049F462E086E00E94590264E086E01F
:101AC0000E94590202C01FBF10C0809132258F3F73
:101AD00009F4FFCF8FB78983F8949981E1E3F5E2A8
:101AE00081818F5F81839FBF1FBF0F900F90DF9118
:101AF000CF911F910895811528E0920729F46093F2
:101B00000E2270930F220895803428E0920729F462
:101B100060930422709305220895811529E09207AD
:101B200029F46093FC217093FD210895803429E00D
:101B3000920729F46093F0217093F12108958115A3
:101B40002AE0920729F46093E8217093E92108952F
:101B500080342AE0920729F46093DC217093DD2120
:101B6000089581152BE0920729F46093D421709396
:101B7000D521089580349B4021F46093C82170934F
:101B8000C9210895CF93DF93E0911022F0911122A3
:101B9000848183FF08C08860848383E0838386EF29
:101BA00080931A2283C0982F947131F083E083834D
:101BB0008FEF80931A227AC086FF43C0C0E1D2E241
:101BC000AA81BB818C819D8114962D913C911597A2
:101BD000821793076CF49C012F5F3F4F20931422D0
:101BE00030931522A80FB91F11968C9187835EC080
:101BF000809116229091172218962D913C91199759
:101C000082179307C8F420911822222321F086819D
:101C1000816086834BC016962D913C911797AC013D
:101C20004F5F5F4F4093162250931722D901A80FA0
:101C3000B91F8C9187833AC083E0838310921A2264
:101C400035C0882384F5A0E1B2E21296CD91DC91F3
:101C5000139716968D919C91179728853985821731
:101C60009307D8F46E817F819C012F5F3F4F2093B3
:101C70001622309317224781DB01A80FB91F4C931E
:101C8000888599852817390718F482E083830EC068
:101C900087E0838310921A2209C083E0838389EF4F
:101CA00080931A2203C08BEF80931A22DF91CF9189
:101CB00008951F920F920FB60F92112408B60F923B
:101CC00018BE09B60F9219BE0BB60F921BBE2F930A
:101CD0003F934F935F936F937F938F939F93AF93B4
:101CE000BF93EF93FF934EDFFF91EF91BF91AF91C1
:101CF0009F918F917F916F915F914F913F912F9124
:101D00000F900BBE0F9009BE0F9008BE0F900FBE34
:101D10000F901F9018951F920F920FB60F921124DB
:101D200008B60F9218BE09B60F9219BE0BB60F92E5
:101D30001BBE2F933F934F935F936F937F938F932C
:101D40009F93AF93BF93EF93FF931CDFFF91EF91AE
:101D5000BF91AF919F918F917F916F915F914F91C3
:101D60003F912F910F900BBE0F9009BE0F9008BEB0
:101D70000F900FBE0F901F9018951F920F920FB6E5
:101D80000F92112408B60F9218BE09B60F9219BE11
:101D90000BB60F921BBE2F933F934F935F936F939E
:101DA0007F938F939F93AF93BF93EF93FF93EADE5D
:101DB000FF91EF91BF91AF919F918F917F916F9123
:101DC0005F914F913F912F910F900BBE0F9009BEE5
:101DD0000F9008BE0F900FBE0F901F9018951F9286
:101DE0000F920FB60F92112408B60F9218BE09B6C3
:101DF0000F9219BE0BB60F921BBE2F933F934F93BA
:101E00005F936F937F938F939F93AF93BF93EF9362
:101E1000FF93B8DEFF91EF91BF91AF919F918F91AA
:101E20007F916F915F914F913F912F910F900BBEDA
:101E30000F9009BE0F9008BE0F900FBE0F901F901D
:101E40001895FC01DB0114968C91858388EB8183C6
:101E500081E08483E0E1F2E211861286E0EAF0E0BC
:101E6000828182608283789480E00895CF93DF93AB
:101E70001F92CDB7DEB79C01FB01892B09F451C03D
:101E8000309709F450C0928580911922882319F067
:101E90009923F1F34AC08FB78983F8948981A0E12F
:101EA000B2E291E019969C93199790E81A969C9348
:101EB0001A978FBF2D933C93119712966D937C9335
:101EC000139714961D921C92159716961D921C92AC
:101ED000179718964C938081880F64817581672BC2
:101EE00011F4411103C0F901868303C08160F90137
:101EF0008683E0E1F2E292859038E9F3F90184818A
:101F00008370813049F0A0E1B2E2ED91FC9111972C
:101F1000848183708130C9F7E0E1F2E28285118625
:101F200005C088EF03C088EF01C086EF0F90DF91F6
:101F3000CF910895FC01918195FFFDCF608380E0F2
:101F400090E00895FC0191819923ECF78081089538
:101F50004F925F926F927F928F929F92AF92BF92B9
:101F6000EF92FF920F931F93CF937C014A015B0185
:101F700028013901FC01848182FF16C0D901C80102
:101F8000689412F8B695A795979587951694D1F70A
:101F9000B901A801032E36E17695679557954795C7
:101FA0003A95D1F7302D15C0D901C801689413F8BE
:101FB000B695A795979587951694D1F7B901A8017D
:101FC000032E37E176956795579547953A95D1F762
:101FD000302D88159905AA05BB0508F4A6C08416FE
:101FE0009506A606B70608F4A2C0F701848182FD13
:101FF00004C0880C991CAA1CBB1CC301B201A5011A
:1020000094010E942D3A2F3F31054105510508F4F6
:1020100090C08FEF90E0A0E0B0E0C9EF05C02817B6
:1020200039074A075B0758F0880F991FAA1FBB1F83
:10203000CD3F0CF48160CF5FC73089F74FC0CC2310
:102040000CF04CC0D501C401880F991FAA1FBB1FFB
:10205000880F991FAA1FBB1F880F991FAA1FBB1F9C
:10206000481A590A6A0A7B0ACE3FF4F48DEF9FEFB3
:102070008C1B9109C7FD939504C0440C551C661C2C
:10208000771C8A95D2F7D501C401B695A795979587
:102090008795BC01CD01640D751D861D971DA50199
:1020A00094010E942D3A37C083E08C0FA501940162
:1020B00004C0220F331F441F551F8A95D2F7DA013F
:1020C000C901B695A79597958795BC01CD01640D7B
:1020D000751D861D971D0E942D3A1DC083E08C0F33
:1020E000A501940104C0220F331F441F551F8A9578
:1020F000D2F7DA01C901B695A79597958795BC01E6
:10210000CD01640D751D861D971D0E942D3A21502D
:10211000310941095109832F8F70C295C07FC82BA7
:10212000F701C783268381E018C080E016C080E0F5
:1021300014C0D501C401880F991FAA1FBB1F880FA7
:10214000991FAA1FBB1F880F991FAA1FBB1F481AE0
:10215000590A6A0A7B0AC9EF89CFCF911F910F9163
:10216000FF90EF90BF90AF909F908F907F906F9077
:102170005F904F9008950F931F93CF93DF93EC01DF
:102180008B01009709F45DC1803C910529F460E161
:1021900080E00E94590255C1C03484E0D80729F478
:1021A00068E080E00E9459024CC1C115E4E0DE07FE
:1021B00029F464E080E00E94590243C1C038F1E094
:1021C000DF0729F462E080E00E9459023AC1C1159C
:1021D00081E0D80729F461E080E00E94590231C112
:1021E000C038E3E0DE0729F461E081E00E94590293
:1021F00028C1C039F3E0DF0729F461E082E00E94E2
:1022000059021FC1C11582E0D80729F462E081E0BC
:102210000E94590216C1C034E2E0DE0729F462E0F0
:1022200082E00E9459020DC1C115F3E0DF0729F4D5
:1022300064E081E00E94590204C1C03283E0D80703
:1022400029F464E082E00E945902FBC0C115E8E075
:10225000DE0729F461E083E00E945902F2C0C11553
:10226000F9E0DF0729F461E084E00E945902E9C047
:10227000C1158AE0D80729F461E085E00E9459027F
:10228000E0C0C115EBE0DE0729F461E086E00E94C2
:102290005902D7C0C034F8E0DF0729F462E083E0D8
:1022A0000E945902CEC0C03489E0D80729F462E008
:1022B00084E00E945902C5C0C034EAE0DE0729F478
:1022C00062E085E00E945902BCC0C034FBE0DF0739
:1022D00029F462E086E00E945902B3C0C03988E068
:1022E000D80729F464E083E00E945902AAC0C039EB
:1022F000E9E0DE0729F464E084E00E945902A1C00D
:10230000C039FAE0DF0729F464E085E00E94590251
:1023100098C0C0398BE0D80729F464E086E00E94B9
:1023200059028FC0C03CE8E0DE0729F468E083E092
:102330000E94590286C0C03CF9E0DF0729F468E03A
:1023400084E00E9459027DC0C03C8AE0D80729F48D
:1023500068E085E00E94590274C0C03CEBE0DE07F3
:1023600029F468E086E00E9459026BC0C03AF8E0A8
:10237000DF0729F460E183E00E94590262C0C03A9D
:1023800089E0D80729F460E184E00E94590259C02D
:10239000C03AEAE0DE0729F460E185E00E945902D4
:1023A00050C0C03AFBE0DF0729F460E186E00E94FC
:1023B000590247C0C03B88E0D80729F460E283E0B7
:1023C0000E9459023EC0C03BE9E0DE0729F460E20A
:1023D00084E00E94590235C0C03BFAE0DF0729F4CF
:1023E00060E285E00E9459022CC0C03B8BE0D80718
:1023F00029F460E286E00E94590223C0C038E4E07C
:10240000DE0729F460E483E00E9459021AC0C03953
:10241000F4E0DF0729F460E484E00E94590211C06F
:10242000C03A84E0D80729F460E485E00E945902AC
:1024300008C0C03BE4E0DE0721F460E486E00E94CF
:1024400059028D818F738D83F80195818481892B49
:102450009681911198E0892B8D83F80140815181FB
:102460006281738100E018E428EE31E0CE0170DD76
:102470009C8198609C839C8190619C83DF91CF912B
:102480001F910F9108959091800024E0829FB001E8
:1024900011246C7392709160692B80E890E00E9427
:1024A0005704E0E8F0E0828180FDFDCF089560915F
:1024B00080006C73636080E890E00E945704E0E85D
:1024C000F0E0828180FDFDCF089563E080E890E038
:1024D0000E945704E0E8F0E0828180FDFDCF6BE2CE
:1024E00081E890E00E945704E0E8F0E0828180FDFE
:1024F000FDCFA895FFCFCF92DF92EF92FF92CF93BF
:10250000DF93EC016B01E12CF12C60E078E488EEC4
:1025100091E0A70196010E942D3ACA01B9012FEF5F
:102520003FEF40E050E00E942D3A2115310529F49B
:1025300081E08C8321E030E02DC02230310528F489
:1025400082E08C8322E030E025C02430310528F47D
:1025500083E08C8324E030E01DC02830310528F46E
:1025600084E08C8328E030E015C02034310528F465
:1025700085E08C8320E430E00DC02F3F310509F069
:1025800028F486E08C8320E031E004C087E08C836F
:1025900020E034E040E050E060E078E488EE91E054
:1025A0000E942D3ACA01B901A70196010E942D3A55
:1025B0002D833E832436310518F41C821D821E8231
:1025C000DF91CF91FF90EF90DF90CF9008950F9320
:1025D0001F93CF93DF93EC018901862F90E0883021
:1025E000910508F09EC0FC018827E250FF4F8F4FF5
:1025F0000C944F3A80E098E088839983E0E4F6E019
:10260000308181E090E02FEF240F02C0880F991FE6
:102610002A95E2F7832B808384C080E498E0888346
:102620009983E0E4F6E0308181E090E023E0240F3C
:1026300002C0880F991F2A95E2F7832B808371C00F
:1026400080E099E088839983E0E6F6E0308181E0DC
:1026500090E02FEF240F02C0880F991F2A95E2F710
:10266000832B80835EC080E499E088839983E0E6D1
:10267000F6E0308181E090E023E0240F02C0880F73
:10268000991F2A95E2F7832B80834BC080E09AE064
:1026900088839983E0E8F6E0308181E090E02FEFD5
:1026A000240F02C0880F991F2A95E2F7832B80839D
:1026B00038C080E49AE088839983E0E8F6E03081CE
:1026C00081E090E023E0240F02C0880F991F2A9533
:1026D000E2F7832B808325C080E09BE08883998389
:1026E000E0EAF6E0308181E090E02FEF240F02C0B5
:1026F000880F991F2A95E2F7832B808312C080E40C
:102700009BE088839983E0EAF6E0308181E090E005
:1027100023E0240F02C0880F991F2A95E2F7832B2C
:1027200080834A83423061F018F4413031F010C0A8
:10273000433049F0443051F00BC080E18B8308C036
:1027400080E28B8305C080E48B8302C080E88B83AA
:102750008881998144D9E881F9818181887F83606A
:1027600081831D821E821C82E881F9818081807FA5
:102770008083B801CE01BFDEDF91CF911F910F9111
:102780000895CF93DF93EC012D813E81A62FB0E019
:102790000E94583A24E630E040E050E00E942D3A92
:1027A0008A81E881F981E6FD17C0823061F018F472
:1027B000813031F01BC0833049F0843051F016C0B5
:1027C00020AF31AF13C022AF33AF10C024AF35AF4D
:1027D0000DC026AF37AF0AC0813019F0823021F02A
:1027E00005C020AF31AF02C022AF33AF8D819E81D3
:1027F000E881F98186A397A38B81E881F981E6FDC1
:1028000004C09181892B818304C091818073892BBD
:102810008183E881F9818081807F9C81892B8083FD
:10282000DF91CF91089510921B2208951F93CF93AB
:10283000DF93162FD42F8C3038F0883139F08C305C
:1028400041F08C5031E006C030E004C030E08CE054
:1028500001C031E0CDEC8C9F412D1124242F269511
:1028600026952695422F440F942F990F990F940F78
:10287000891B982F9064832F8295880F807E892BE7
:1028800090E1299FA0011124482B62E088E60E9474
:10289000692F1C9F812D112486958695869590E140
:1028A000899FA0011124880F982F990F990F890FE4
:1028B000181B412B61E088E60E94692FDC9FC12D27
:1028C0001124C695C695C69580E1C89FA001112424
:1028D000CC0F8C2F880F880FC80FDC1B4D2B60E0AE
:1028E00088E60E94692FDF91CF911F910895109281
:1028F0001B2240E06EE088E60E94692F40E06FE016
:1029000088E60E94692FE0E6F6E082E0808B81E0B5
:10291000838781858C60818740E06AE383E086CF8E
:102920000895CF93DF93EC012CE132E243E060E0C5
:1029300088E60E947A2FECE1F2E222819181808187
:1029400024FB332730F9330F432F440F440F340F48
:10295000422F4F70340F3883392F36953695369580
:102960003E71432F440F440F340F9F70930F998390
:10297000982F9695969596959E71392F330F330F14
:10298000930F8F70890F8A8325FB222720F92B83D1
:10299000DF91CF91089580911B2208951F920F928D
:1029A0000FB60F92112408B60F9218BE8F9381E0D4
:1029B00080931B228F910F9008BE0F900FBE0F9037
:1029C0001F901895FC011282A081B1811C9282E0B7
:1029D000838308950F931F93CF93DF9388E190E251
:1029E0000E94E22E9F938F938EE190E29F938F93AC
:1029F00088E08F9380EA8F93E0913D25F0913E250A
:102A00001995CCE3D2E204E612E20F900F900F90FA
:102A10000F900F900F90CE01D5DF2496C017D107ED
:102A2000D1F7E6E4F9E280E895E2A0E0B0E0808347
:102A30009183A283B38381E08683158283E08483BC
:102A4000BF0180EB98E097DB82E290E29F938F9347
:102A5000D8E0DF93C0EBCF93E0913D25F0913E2588
:102A6000199585E390E29F938F93DF93CF93E09145
:102A70003D25F0913E25199586E490E29F938F9332
:102A8000DF93CF93E0913D25F0913E2519958AE79C
:102A900090E29F938F93DF93CF93E0913D25F09148
:102AA0003E25199584E990E29F938F93DF93CF930E
:102AB000E0913D25F0913E251995E0EBF8E083810A
:102AC0008F7C806283838DB79EB744968DBF9EBFF7
:102AD000DF91CF911F910F9108951F920F920FB622
:102AE0000F92112408B60F9218BE09B60F9219BEA4
:102AF0000BB60F921BBE2F933F934F935F936F9331
:102B00007F938F939F93AF93BF93EF93FF9380EB4C
:102B100098E018DA80934529FF91EF91BF91AF912A
:102B20009F918F917F916F915F914F913F912F91E5
:102B30000F900BBE0F9009BE0F9008BE0F900FBEF6
:102B40000F901F90189504C0615071098109910977
:102B50006115710581059105B9F7089548E066E6AC
:102B600072E286EA92E20E949D2D48E066E872E2F7
:102B70008BEA92E20E949D2D1092652210926422AF
:102B800044E066E280E60E94692F2BEB32E241E0EE
:102B900066E280E60E947A2F8091BB2282FDF5CF0B
:102BA00047E063E180E60E94692F40E268E280E648
:102BB0000E94692F40E869E280E60E94692F40E8A0
:102BC0006AE280E60E94692F48E966E280E60E9498
:102BD000692F66E573E288E090E0B5DFE0E6F6E0B5
:102BE00081E3828B84E08287818583608187089579
:102BF000CF93DF93209164222223E1F0EC018BEA52
:102C000092E20E94F82C6D837E838F83988786EAF8
:102C100092E20E94F82C2091B1223091B222409190
:102C2000B3225091B4220E94D33169837A838B837B
:102C30009C8309C0FC0111821282138214821582C6
:102C4000168217821086DF91CF91089580916522B8
:102C50000895811106C04AE866E280E60C94692F67
:102C600008954AE066E280E60C94692F0895CF92B9
:102C7000DF92EF92FF92CF93DF93C0EBD2E26985B0
:102C80007A85072E000C880B990B0E9450336B013C
:102C90007C019B01AC0169817A818B819C810E94BE
:102CA000B53269837A838B839C83A70196016D81FA
:102CB0007E818F8198850E94B5326D837E838F835C
:102CC000988721E030E029873A87209364220E9488
:102CD0005C308C818F938B818F938A818F938981D4
:102CE0008F9386EA90E29F938F9388E08F9380EA98
:102CF0008F93E0913D25F0913E2519958DB79EB7B4
:102D000008968DBF9EBFDF91CF91FF90EF90DF902F
:102D1000CF9008958F929F92AF92BF92CF92DF9201
:102D2000EF92FF920F931F93CF93DF931092652240
:102D30002BEB32E246E060E080E60E947A2F809141
:102D4000BB2283FFDAC0CBEBD2E2B980CA80AB8072
:102D50001C810D819E0141E066E280E60E947A2F8F
:102D6000888188231CF56C2D70E07B29072E000CD0
:102D7000880B990B0E9450336B017C01CA2DC295C0
:102D8000CF706C2F70E080E090E00E94503320E024
:102D900030E040E85DE30E94A1349B01AC01C70133
:102DA000B6010E94D4316B017C012FC0D12CE12CE3
:102DB000F12CFE2CED2CDC2CCC24EB28CA28CA2DBF
:102DC000C073C295CF706C2F70E080E090E00E94DD
:102DD0004E3320E030E040E85EE30E94A1344B0136
:102DE0005C01C701B601689415F8959587957795AC
:102DF00067951694D1F70E9450339B01AC01C50131
:102E0000B4010E94D4316B017C01A7019601C70176
:102E1000B6010E94B535811172C020E030E0A901F1
:102E2000C701B6010E94B132882309F46AC0D02FCD
:102E3000D295DF706D2F70E080E090E00E945033FB
:102E400020E030E040E85DE30E94A1344B015C01EA
:102E5000612F70E080E090E00E944E339B01AC0156
:102E6000C501B4010E94D4314B015C019B01AC014E
:102E70000E94B535811147C020E030E0A901C501AD
:102E8000B4010E94B132882309F43FC0C09164228A
:102E9000CC2369F0B501A4018BEA92E20E94CE2C0A
:102EA000B701A60186EA92E20E94CE2C31C0C0EBA7
:102EB000D2E2A701960169817A818B819C810E946F
:102EC000D43169837A838B839C83A50194016D81BE
:102ED0007E818F8198850E94D4316D837E838F831C
:102EE000988789859A85019689879A878038910580
:102EF00074F0CE01BCDEC1E00BC0C0E009C0C0E090
:102F000007C0C0E005C0C0E003C0C0E001C0C1E030
:102F10008C2FDF91CF911F910F91FF90EF90DF9059
:102F2000CF90BF90AF909F908F9008951F920F9277
:102F30000FB60F92112408B60F9218BE8F9381E03E
:102F4000809365228F910F9008BE0F900FBE0F9057
:102F50001F90189504C0615071098109910961158C
:102F6000710581059105B9F7089580938924089525
:102F7000809189240895682F70E088EE93E00E9484
:102F8000063A4FEF460F69E189E60C94692F0895E0
:102F9000CF93DF93EC0184E494E20E94F82C6883E1
:102FA00079838A839B8387E194E20E94F82C6C8367
:102FB0007D838E839F838AEE93E20E94F82C68873C
:102FC00079878A879B87DF91CF910895CF93DF938D
:102FD000EC018DEB93E20E94CD2D688379838A8387
:102FE0009B8380E993E20E94CD2D6C837D838E8349
:102FF0009F8383E693E20E94CD2D688779878A8735
:103000009B87DF91CF9108952F923F924F925F92CD
:103010006F927F928F929F92AF92BF92CF92DF92E8
:10302000EF92FF920F931F93CF93DF93CDB7DEB74D
:10303000A497CDBFDEBFFC01A080B180C280D38049
:10304000E488F5880689178920893189428953895E
:10305000448455846684778480A191A1A2A1B3A100
:10306000B058BF93AF939F938F93878D8F93868D27
:103070008F93858D8F93848D8F93838D8F93828D86
:103080008F93818D8F93808D8F9383858F9382858E
:103090008F9381858F9380858F9387818F9386818E
:1030A0008F9385818F9384818F93C301B2010E9496
:1030B0002224609100207091012080910220909143
:1030C0000320209100203091012040910220509156
:1030D00003208090A4249090A524A090A624B090D2
:1030E000A7244090A4245090A5246090A62470901A
:1030F000A724E090A024F090A1240091A224109194
:10310000A324E982FA820B831C83E090A024F09030
:10311000A1240091A2241091A324ED82FE820F83AA
:103120001887E0909C24F0909D2400919E2410919B
:103130009F24E986FA860B871C87E0909C24F090F8
:103140009D2400919E2410919F24ED86FE860F877A
:10315000188BE090A424F090A5240091A62410914F
:10316000A724E98AFA8A0B8B1C8BE090A024F090AC
:10317000A1240091A2241091A324ED8AFE8A0F8B32
:10318000188FE0900020F090012000910220109113
:103190000320E9A2FAA20BA31CA3E0909C24F090C8
:1031A0009D2400919E2410919F24E98EFA8E0B8F0E
:1031B0001C8F0E94A1346B017C01A3019201C50107
:1031C000B4010E94A1349B01AC01C701B6010E9469
:1031D000D4314B015C012D813E814F81588569813D
:1031E0007A818B819C810E94A1349B01AC01C50135
:1031F000B4010E94D3314B015C012D853E854F8582
:10320000588969857A858B859C850E94A1349B01AC
:10321000AC01C501B4010E94D3312B013C012D89C1
:103220003E894F89588D69897A898B899C890E944A
:10323000A1344B015C01298D3A8D4B8D5C8D69A1C8
:103240007AA18BA19CA10E94A1349B01AC01C50174
:10325000B4010E94D4319B01AC010E94D431A3017E
:1032600092010E945E320F2EF6E72F2EF9E23F2EDA
:10327000F02DF10160837183828393836091A42494
:103280007091A5248091A6249091A72420919C243C
:1032900030919D2440919E2450919F248090002045
:1032A00090900120A0900220B09003204090A02494
:1032B0005090A1246090A2247090A3240E94A13475
:1032C0006B017C01A3019201C501B4010E94A134EC
:1032D0009B01AC01C701B6010E94D3319B01AC0137
:1032E0000E94D4310E943832DC01CB01B058809367
:1032F0007A2990937B29A0937C29B0937D296091B2
:103300000020709101208091022090910320209153
:1033100000203091012040910220509103208090A4
:10332000A4249090A524A090A624B090A724409017
:10333000A4245090A5246090A6247090A724E09027
:10334000A024F090A1240091A2241091A324E9824A
:10335000FA820B831C83E090A024F090A1240091BA
:10336000A2241091A324ED82FE820F831887E0909F
:103370009C24F0909D2400919E2410919F24E98626
:10338000FA860B871C87E0909C24F0909D24009186
:103390009E2410919F24ED86FE860F87188BE09067
:1033A0000020F09001200091022010910320E98A72
:1033B000FA8A0B8B1C8BE090A424F090A52400913A
:1033C000A6241091A724ED8AFE8A0F8B188FE09017
:1033D000A024F090A1240091A2241091A324E9A29A
:1033E000FAA20BA31CA3E0909C24F0909D240091D2
:1033F0009E2410919F24E98EFA8E0B8F1C8F0E94C1
:10340000A1346B017C01A3019201C501B4010E94AA
:10341000A1349B01AC01C701B6010E94D3314B011D
:103420005C012D813E814F81588569817A818B8134
:103430009C810E94A1349B01AC01C501B4010E9492
:10344000D3314B015C012D853E854F8558896985B7
:103450007A858B859C850E94A1349B01AC01C501B6
:10346000B4010E94D4312B013C012D893E894F8942
:10347000588D69897A898B899C890E94A1344B0176
:103480005C01298D3A8D4B8D5C8D69A17AA18BA150
:103490009CA10E94A1349B01AC01C501B4010E9412
:1034A000D4319B01AC010E94D431A30192010E944E
:1034B0005E3260937E2970937F2980938029909358
:1034C000812960917A2970917B2980917C29909142
:1034D0007D292DEE3EE245E652E40E94A134609340
:1034E0007A2970937B2980937C2990937D29F1011F
:1034F00060817181828193812DEE3EE245E652E446
:103500000E94A134F101608371838283938360916F
:103510007E2970917F2980918029909181292DEEBB
:103520003EE245E652E40E94A13460937E29709306
:103530007F298093802990938129F10140815181D5
:10354000628173818DEB93E20E94A32D40917A29D1
:1035500050917B2960917C2970917D2980E993E2CB
:103560000E94A32D40917E2950917F29609180294E
:103570007091812983E693E20E94A32DCDBFDEBF27
:10358000A496CDBFDEBFDF91CF911F910F91FF9029
:10359000EF90DF90CF90BF90AF909F908F907F90F3
:1035A0006F905F904F903F902F900895CF92DF9251
:1035B000EF92FF920F931F93CF93DF9329E434E2AE
:1035C0004FE06AE389E60E947A2F8091492480FFC8
:1035D00032C1E9E4F4E2818190E0982F88272281CA
:1035E000822B0EE819E2D8018D939C931197838169
:1035F00090E0982F88272481822B12968D939C939C
:103600001397858190E0982F88272681822B149626
:103610008D939C931597818590E0982F882722851C
:10362000822B16968D939C931797838590E0982F05
:1036300088272485822B18968D939C9319978585CE
:1036400090E0982F88272685822B1A968D939C933D
:103650001B976D917C91C0908A29D0908B29E09026
:103660008C29F0908D29072E000C880B990B0E9455
:103670005033A70196010E94A134C2E5D9E26883C4
:1036800079838A839B83F80162817381C0908A2940
:10369000D0908B29E0908C29F0908D29072E000C7A
:1036A000880B990B0E945033A70196010E94A13408
:1036B0006C837D838E839F83D80114966D917C915A
:1036C0001597C0908A29D0908B29E0908C29F09092
:1036D0008D29072E000C880B990B0E945033A701EF
:1036E00096010E94A134688779878A879B87F801B1
:1036F00066817781C0908629D0908729E0908829BB
:10370000F0908929072E000C880B990B0E945033EA
:10371000A70196010E94A1346C877D878E879F87C1
:10372000D80118966D917C911997C0908629D090F8
:103730008729E0908829F0908929072E000C880BB2
:10374000990B0E945033A70196010E94A134688B07
:10375000798B8A8B9B8BF80162857385C090862953
:10376000D0908729E0908829F0908929072E000CB5
:10377000880B990B0E945033A70196010E94A13437
:103780006C8B7D8B8E8B9F8B188E198E1A8E1B8E59
:103790001C8E1D8E1E8E1F8E18A219A21AA21BA28D
:1037A000088519852A853B854C815D816E817F81E5
:1037B00088819981AA81BB813F932F931F930F9397
:1037C0007F936F935F934F93BF93AF939F938F9329
:1037D0008AEB90E29F938F9388E08F9380EA8F9398
:1037E000E0913D25F0913E251995488159816A81E6
:1037F0007B8184E494E20E94CE2C4C815D816E81B9
:103800007F8187E194E20E94CE2C488559856A85A4
:103810007B858AEE93E20E94CE2CCE01F5DB29E473
:1038200034E241E06AE389E60E947A2F8DB79EB7C1
:1038300040968DBF9EBFDF91CF911F910F91FF905A
:10384000EF90DF90CF90089529E434E241E065E7FE
:1038500089E60E947A2F80914924813789F480ED8E
:1038600090E29F938F9388E08F9380EA8F93E0910B
:103870003D25F0913E2519950F900F900F900F90D8
:103880000895813099F028F08230E9F0833041F1D9
:1038900033C080E090E0A0E8B8E380938A29909359
:1038A0008B29A0938C29B0938D2926C080E090E0CD
:1038B000A0E0B9E380938A2990938B29A0938C2967
:1038C000B0938D2919C080E090E0A0E8B9E380931F
:1038D0008A2990938B29A0938C29B0938D290CC0B1
:1038E00080E090E0A0E0BAE380938A2990938B294E
:1038F000A0938C29B0938D2948E16CE189E60C9462
:10390000692F0895813099F028F08230E9F08330F2
:1039100041F133C081EA9FE0AAEFBBE3809386299F
:1039200090938729A0938829B093892926C081EA9A
:103930009FE0AAE7BCE38093862990938729A09310
:103940008829B093892919C081EA9FE0AAEFBCE3D6
:103950008093862990938729A0938829B0938929F9
:103960000CC080E090E0AAE7BDE3809386299093A5
:103970008729A0938829B093892948E16BE189E6DA
:103980000C94692F08954AE065E973E28DEB93E2A8
:103990000E94722E4AE068E673E280E993E20E9498
:1039A000722E4AE06BE373E283E693E20E94722E8A
:1039B0004AE06CE174E284E494E20E949D2D4AE0C6
:1039C0006FEE73E287E194E20E949D2D4AE062EC83
:1039D00073E28AEE93E20E949D2D40E86BE689E651
:1039E0000E94692F66E573E288E090E0B3DA41E077
:1039F0006BE689E60E94692F40E06CE689E60E944A
:103A0000692F66E573E288E090E0A4DA42E06AE1BB
:103A100089E60E94692F83E075DF83E032DF42E0B0
:103A20006DE189E60E94692F84E6A5DA42E267E348
:103A300089E60E94692F41E068E389E60E94692FC8
:103A4000E0E0F6E081E1828B84E0828783E0818799
:103A500008951F920F920FB60F92112408B60F927D
:103A600018BE8F9381E0809389248F910F9008BEB8
:103A70000F900FBE0F901F901895E0E0F2E080A12C
:103A8000806880A30895F9DFE0E0F2E083A1882355
:103A9000E9F3E0E0F2E084A195A1168208958F9207
:103AA0009F92AF92BF92CF92DF92EF92FF92CF930D
:103AB000C42F0E944E3320E030E44CE156E40E94D3
:103AC000B5320E9461346B017C019B01AC010E9404
:103AD000D43122E835ED4FE256E30E94A1344B0188
:103AE0005C0121EF3BEB46E859E3C701B6010E94B8
:103AF000A1342DE03FEC4BE55BE30E94D4319B0108
:103B0000AC01C501B4010E94D4314B015C0120E03D
:103B100030E040E450E4C701B6010E94A1342AE637
:103B200033E149E853E30E94A1349B01AC01C50194
:103B3000B4010E94D4319B01AC0160E070E080E8E8
:103B40009FE30E94B532CC2389F023E333E948E8B0
:103B500053E4C62ED72EE82EF92EC701B6010E94D7
:103B6000D331562F472F382F292F04C0562F472FD8
:103B7000382F292F652F742F832F922FCF91FF90ED
:103B8000EF90DF90CF90BF90AF909F908F9008956F
:103B9000EAE8F4E210821182128213821482158202
:103BA0000895FF920F931F93CF93DF938C01F62E0E
:103BB000CAE8D4E26C817D81072E000C880B990B3A
:103BC0000E9450339B01AC01688179818A819B817D
:103BD0000E94B532F8016083718382839383F11070
:103BE000D7DFDF91CF911F910F91FF9008954F92F2
:103BF0005F926F927F928F929F92AF92BF92CF927D
:103C0000DF92EF92FF920F931F93CF93DF938C017C
:103C1000181619060CF040C0C0E0D0E0812C912CA1
:103C2000540131DFBC0180E090E00E944E3320E07F
:103C300030E044E050E40E94A13420E030E040E86D
:103C400059E30E94A1346B017C0120E030E24BE497
:103C500056E40E94A1342B013C01A701960163E3C5
:103C600073E383E590E40E94D3319B01AC01C3016F
:103C7000B2010E94B5320E94223341E010DF9B0165
:103C8000AC01C501B4010E94D4314B015C01219605
:103C90000C171D0731F603C0812C912C5401B8017B
:103CA000110F880B990B0E9450339B01AC01C50189
:103CB000B4010E94B532DF91CF911F910F91FF9017
:103CC000EF90DF90CF90BF90AF909F908F907F90BC
:103CD0006F905F904F90089584E090E088DF20918E
:103CE000A0293091A1294091A2295091A3290C9497
:103CF000D3310895CF93DF931092A0291092A12978
:103D00001092A2291092A329E0E0F2E081E080A3C2
:103D100011A2C0913D25D0913E25DEDF9F938F9368
:103D20007F936F938CEE90E29F938F9388E08F93B5
:103D300080EA8F93FE0119958DB79EB708968DBFC7
:103D40009EBFDF91CF9108950F931F93CF93DF9381
:103D500000E012E081E0F8018083118280E182833B
:103D600085E0848361E270E082E00E945D04C82FF8
:103D7000D0E0DC2FCC2760E270E082E00E945D049E
:103D8000C82BF801C487D587DF91CF911F910F9180
:103D900008954F925F926F927F928F929F92AF920F
:103DA000BF92CF92DF92EF92FF920F931F93CF9328
:103DB000DF93CDB7DEB7A497CDBFDEBF69877A8723
:103DC0008B879C872D873E874F87588BE98AFA8A95
:103DD0000B8B1C8B20E030E0A901C601B5010E94CD
:103DE000B132811117C020E030E0A90168AD79AD92
:103DF0008AAD9BAD0E94B13281110CC020E030E051
:103E0000A9016CAD7DAD8EAD9FAD0E94B13288230E
:103E100009F489C2A6019501C601B5010E94A13429
:103E20002B013C0128AD39AD4AAD5BADCA01B901EA
:103E30000E94A1349B01AC01C301B2010E94D431A4
:103E40002B013C012CAD3DAD4EAD5FADCA01B901BA
:103E50000E94A1349B01AC01C301B2010E94D43184
:103E60002B013C0175946794579447941FEDE12E04
:103E700019E5F12E07E31FE5E418F508060917090F
:103E800020E030E040E05FE30E94A134A801970108
:103E90000E94A134A80197010E94A1349B01AC01AA
:103EA00060E070E080EC9FE30E94D331A8019701AD
:103EB0000E94A1342B013C019B01AC01C601B5015C
:103EC0000E94A13469837A838B839C83A30192012E
:103ED00068AD79AD8AAD9BAD0E94A1346D837E83C0
:103EE0008F839887A30192016CAD7DAD8EAD9FADA0
:103EF0000E94A1346D8B7E8B8F8B988F6091A42450
:103F00007091A5248091A6249091A72420919C24AF
:103F100030919D2440919E2450919F2480900020B8
:103F200090900120A0900220B09003204090A02407
:103F30005090A1246090A2247090A3240E94A134E8
:103F40006B017C01A3019201C501B4010E94A1345F
:103F50009B01AC01C701B6010E94D331698F7A8FF2
:103F60008B8F9C8F609100207091012080910220A6
:103F7000909103202091A4243091A5244091A6245F
:103F80005091A7248090A0249090A124A090A224D6
:103F9000B090A32440909C2450909D2460909E2437
:103FA00070909F240E94A1346B017C01A3019201B7
:103FB000C501B4010E94A1349B01AC01C701B60147
:103FC0000E94D4316D8F7E8F8F8F98A360910020D7
:103FD0007091012080910220909103202091002077
:103FE00030910120409102205091032080909C2428
:103FF00090909D24A0909E24B0909F2440909C245B
:1040000050909D2460909E2470909F240E94A13423
:1040100020E030E040E05FE30E94D3316B017C019F
:10402000A3019201C501B4010E94A1349B01AC011E
:10403000C701B6010E94D4316B017C019B01AC0128
:104040006D817E818F8198850E94A1344B015C0136
:104050002D8D3E8D4F8D58A16D897E898F89988DCC
:104060000E94A1349B01AC01C501B4010E94D3316F
:1040700069A37AA38BA39CA3298D3A8D4B8D5C8D6C
:104080006D897E898F89988D0E94A1344B015C01D6
:10409000A701960169817A818B819C810E94A1345C
:1040A0009B01AC01C501B4010E94D3314B015C01FD
:1040B0002D8D3E8D4F8D58A169817A818B819C8198
:1040C0000E94A1346B017C01298D3A8D4B8D5C8D52
:1040D0006D817E818F8198850E94A1349B01AC0106
:1040E000C701B6010E94D3316B017C016091A82405
:1040F0007091A9248091AA249091AB2420E030E013
:10410000A9010E94513418160CF0ABC02091A824CC
:104110003091A9244091AA245091AB244090982436
:104120005090992460909A2470909B2469A17AA160
:104130008BA19CA10E94A1342AEF39EC44E359E3FE
:104140000E94A134A30192010E94D431609398246B
:104150007093992480939A2490939B242091A8246F
:104160003091A9244091AA245091AB2440909424EA
:10417000509095246090962470909724C501B401C6
:104180000E94A1342AEF39EC44E359E30E94A134A0
:10419000A30192010E94D4316093942470939524DA
:1041A00080939624909397242091A8243091A92459
:1041B0004091AA245091AB24409090245090912497
:1041C0006090922470909324C701B6010E94A1349C
:1041D0002AEF39EC44E359E30E94A134A301920190
:1041E0000E94D43160939024709391248093922400
:1041F00090939324209198243091992440919A246B
:1042000050919B2469857A858B859C850E94D43149
:1042100069877A878B879C87209194243091952495
:1042200040919624509197246D857E858F8598893D
:104230000E94D4316D877E878F87988B2091902440
:1042400030919124409192245091932469897A89E4
:104250008B899C890E94D431698B7A8B8B8B9C8B48
:1042600018C0109298241092992410929A241092B7
:104270009B241092942410929524109296241092CC
:1042800097241092902410929124109292241092CC
:1042900093242091042030910520409106205091D4
:1042A000072069A17AA18BA19CA10E94A1349B0146
:1042B000AC0169857A858B859C850E94D43169879C
:1042C0007A878B879C87209104203091052040912C
:1042D000062050910720C501B4010E94A1349B0122
:1042E000AC016D857E858F8598890E94D4316D875C
:1042F0007E878F87988B20910420309105204091F4
:10430000062050910720C701B6010E94A1349B01ED
:10431000AC0169897A898B899C890E94D431698B27
:104320007A8B8B8B9C8B2AEF39EC44EB58E36985B5
:104330007A858B859C850E94A13469877A878B87D3
:104340009C872AEF39EC44EB58E36D857E858F8599
:1043500098890E94A1346D877E878F87988B2AEF7A
:1043600039EC44EB58E369897A898B899C890E94EE
:10437000A134698B7A8B8B8B9C8BE0900020F09022
:1043800001200091022010910320ED82FE820F8314
:1043900018878090A4249090A524A090A624B09083
:1043A000A724E090A024F090A1240091A2241091D1
:1043B000A324ED8AFE8A0F8B188F40909C24509086
:1043C0009D2460909E2470909F24C0900020D090E7
:1043D0000120E0900220F0900320C501B401905824
:1043E00029853A854B855C850E94A13469837A834F
:1043F0008B839C832D893E894F89588D6D857E8561
:104400008F8598890E94A1349B01AC0169817A81D2
:104410008B819C810E94D33169837A838B839C83B7
:10442000A301920169897A898B899C890E94A134B0
:104430009B01AC0169817A818B819C810E94D3317F
:10444000A70196010E94D43160930020709301204F
:10445000809302209093032040909C2450909D24B0
:1044600060909E2470909F24C090A424D090A52496
:10447000E090A624F090A7242D813E814F8158859D
:1044800069857A858B859C850E94A13469837A83AE
:104490008B839C832D893E894F89588D69897A89C0
:1044A0008B899C890E94A1349B01AC0169817A812E
:1044B0008B819C810E94D43169837A838B839C8316
:1044C000A30192016D857E858F8598890E94A13414
:1044D0009B01AC0169817A818B819C810E94D331DF
:1044E000A70196010E94D4316093A4247093A5245F
:1044F0008093A6249093A72440909C2450909D24C0
:1045000060909E2470909F24C090A024D090A124FD
:10451000E090A224F090A3242D813E814F81588504
:104520006D857E858F8598890E94A13469837A8301
:104530008B839C83A501940169897A898B899C89E5
:104540000E94A1349B01AC0169817A818B819C819D
:104550000E94D33169837A838B839C83A301920168
:1045600069857A858B859C850E94A1349B01AC016D
:1045700069817A818B819C810E94D431A701960147
:104580000E94D4316093A0247093A1248093A2242C
:104590009093A324C0909C24D0909D24E0909E24CE
:1045A000F0909F242D813E814F81588569897A89B9
:1045B0008B899C890E94A1342B013C01A5019401A7
:1045C0006D857E858F8598890E94A1349B01AC0101
:1045D000C301B2010E94D4314B015C012D893E8997
:1045E0004F89588D69857A858B859C850E94A13479
:1045F0009B01AC01C501B4010E94D331A701960112
:104600000E94D43160939C2470939D2480939E24B7
:1046100090939F246091002070910120809102204E
:1046200090910320209100203091012040910220A0
:10463000509103208090A4249090A524A090A624BB
:10464000B090A7244090A4245090A5246090A62464
:104650007090A724E090A024F090A1240091A224BF
:104660001091A324E986FA860B871C87E090A0248A
:10467000F090A1240091A2241091A324ED86FE863F
:104680000F87188BE0909C24F0909D2400919E242D
:1046900010919F24E982FA820B831C83E0909C2472
:1046A000F0909D2400919E2410919F24E98AFA8A1B
:1046B0000B8B1C8B0E94A1346B017C01A301920126
:1046C000C501B4010E94A1349B01AC01C701B60130
:1046D0000E94D4314B015C012D853E854F85588960
:1046E00069857A858B859C850E94A1349B01AC01EC
:1046F000C501B4010E94D4314B015C0129893A897A
:104700004B895C8969817A818B819C810E94A1346B
:104710009B01AC01C501B4010E94D4314B015C0185
:10472000B594A794979487940F2EFFEDCF2EF9E5BB
:10473000DF2EF7E3EF2EFFE5FF2EF02DC818D90886
:10474000EA08FB0820E030E040E05FE30E94A1348B
:10475000A70196010E94A134A70196010E94A134ED
:104760009B01AC0160E070E080EC9FE30E94D331DC
:10477000A70196010E94A1346B017C016091002089
:10478000709101208091022090910320A701960151
:104790000E94A13460930020709301208093022036
:1047A000909303206091A4247091A5248091A62465
:1047B0009091A724A70196010E94A1346093A4249C
:1047C0007093A5248093A6249093A7246091A0249D
:1047D0007091A1248091A2249091A324A701960115
:1047E0000E94A1346093A0247093A1248093A224FA
:1047F0009093A32460919C2470919D2480919E2489
:1048000090919F24A70196010E94A13460939C245B
:1048100070939D2480939E2490939F24A496CDBF53
:10482000DEBFDF91CF911F910F91FF90EF90DF904E
:10483000CF90BF90AF909F908F907F906F905F9040
:104840004F9008952F923F924F925F926F927F9276
:104850008F929F92AF92BF92CF92DF92EF92FF9290
:104860000F931F93CF93DF93CDB7DEB7C855D10910
:10487000CDBFDEBF698B7A8B8B8B9C8B298F3A8F58
:104880004B8F5C8FE982FA820B831C83AF96FFAC5F
:10489000AF97E096EFACE097E1969FACE197E29698
:1048A0008FACE297E3961FADE397E4960FADE497E4
:1048B000E5963FACE597E6962FACE69720E030E032
:1048C000A901EA966CAD7DAD8EAD9FADEA970E94D1
:1048D000B132811135C020E030E0A901EE966CAD17
:1048E0007DAD8EAD9FADEE970E94B132811128C093
:1048F00020E030E0A901C258DF4F688179818A81C8
:104900009B81CE57D0400E94B132811119C02F92A5
:104910003F920F931F938F929F92EF92FF92E980A5
:10492000FA800B811C81298D3A8D4B8D5C8D6989B4
:104930007A898B899C892DDACDBFDEBF0C94B32C8C
:1049400020E030E0A901C601B5010E94B132811119
:1049500017C020E030E0A9016F2D7E2D892D982D04
:104960000E94B13281110CC020E030E0A901612F1A
:10497000702F832D922D0E94B132882309F489C5AE
:10498000A6019501C601B5010E94A1342B013C018D
:104990002F2D3E2D492D582D6F2D7E2D892D982D93
:1049A0000E94A1349B01AC01C301B2010E94D43129
:1049B0002B013C01212F302F432D522D612F702FC1
:1049C000832D922D0E94A1349B01AC01C301B20141
:1049D0000E94D4312B013C017594679457944794FD
:1049E0002FED39E547E35FE52419350946095709F5
:1049F00029013A0120E030E040E05FE30E94A13469
:104A0000A30192010E94A134A30192010E94A1344A
:104A10009B01AC0160E070E080EC9FE30E94D33129
:104A2000A30192010E94A1342B013C019B01AC0126
:104A3000C601B5010E94A1346DAB7EAB8FAB98AFC0
:104A4000A30192016F2D7E2D892D982D0E94A134F6
:104A500069AF7AAF8BAF9CAFA3019201612F702F2A
:104A6000832D922D0E94A13421966CAF7DAF8EAF25
:104A70009FAF2197EA962CAD3DAD4EAD5FADEA9765
:104A8000CA01B9010E94A1346B017C01EE962CADE4
:104A90003DAD4EAD5FADEE97CA01B9010E94A134A4
:104AA0009B01AC01C701B6010E94D4316B017C01AE
:104AB000C258DF4F288139814A815B81CE57D0406F
:104AC000CA01B9010E94A1349B01AC01C701B60122
:104AD0000E94D4318B019C01359527951795079538
:104AE0000F2EFFEDCF2EF9E5DF2EF7E3EF2EFFE5DA
:104AF000FF2EF02DC01AD10AE20AF30A20E030E0BE
:104B000040E05FE30E94A134A70196010E94A13416
:104B1000A70196010E94A1349B01AC0160E070E006
:104B200080EC9FE30E94D331A70196010E94A1343B
:104B30006B017C019B01AC01EA966CAD7DAD8EAD45
:104B40009FADEA970E94A1346D837E838F839887FF
:104B5000A7019601EE966CAD7DAD8EAD9FADEE9743
:104B60000E94A13469877A878B879C87A701960169
:104B7000C258DF4F688179818A819B81CE57D040AE
:104B80000E94A1346D877E878F87988B409000208C
:104B9000509001206090022070900320E09000204F
:104BA000F090012000910220109103206996ECAE54
:104BB000FDAE0EAF1FAF699760910020709101208C
:104BC00080910220909103202091A4243091A5246B
:104BD0004091A6245091A7240E94A13469A37AA3EE
:104BE0008BA39CA3609100207091012080910220F2
:104BF000909103202091A0243091A1244091A224DF
:104C00005091A3240E94A1346D8F7E8F8F8F98A323
:104C100060910020709101208091022090910320EA
:104C200020919C2430919D2440919E2450919F245A
:104C30000E94A1346D8B7E8B8F8B988FC090A424A3
:104C4000D090A524E090A624F090A7240091A4245D
:104C50001091A5242091A6243091A72409AB1AAB6A
:104C60002BAB3CAB6091A4247091A5248091A62429
:104C70009091A7242091A0243091A1244091A224B6
:104C80005091A3240E94A13469A77AA78BA79CA75F
:104C90006091A4247091A5248091A6249091A724CA
:104CA00020919C2430919D2440919E2450919F24DA
:104CB0000E94A1346DA77EA78FA798AB6091A02416
:104CC0007091A1248091A2249091A3242091A024EA
:104CD0003091A1244091A2245091A3240E94A13498
:104CE00025966CAF7DAF8EAF9FAF25976091A024C6
:104CF0007091A1248091A2249091A32420919C24BE
:104D000030919D2440919E2450919F240E94A13473
:104D100029966CAF7DAF8EAF9FAF299760919C2491
:104D200070919D2480919E2490919F2420919C2499
:104D300030919D2440919E2450919F240E94A13443
:104D40006DA37EA38FA398A725962CAD3DAD4EAD48
:104D50005FAD259760E070E080E09FE30E94D33173
:104D60002DA13EA14FA158A50E94D3312D966CAF25
:104D70007DAF8EAF9FAF2D972D893E894F89588D7E
:104D800069A57AA58BA59CA50E94D33161966CAFCD
:104D90007DAF8EAF9FAF61972DA53EA54FA558A9BA
:104DA0006D8D7E8D8F8D98A10E94D43165966CAFEC
:104DB0007DAF8EAF9FAF65972D962CAD3DAD4EADBF
:104DC0005FAD2D976D817E818F8198850E94A13482
:104DD0004B015C0161962CAD3DAD4EAD5FAD619771
:104DE00069857A858B859C850E94A1349B01AC01E5
:104DF000C501B4010E94D4314B015C0165962CAD14
:104E00003DAD4EAD5FAD65976D857E858F8598898B
:104E10000E94A1349B01AC01C501B4010E94D431B0
:104E20009B01AC010E94D4314B015C0129A93AA934
:104E30004BA95CA9C701B6010E94A1349B01AC013A
:104E400060E070E080E09FE30E94D33169AB7AAB11
:104E50008BAB9CAB29A53AA54BA55CA56D897E893A
:104E60008F89988D0E94D4312D813E814F81588544
:104E70000E94A1346B017C012DA13EA14FA158A538
:104E800069A97AA98BA99CA90E94D33129853A8561
:104E90004B855C850E94A1349B01AC01C701B60122
:104EA0000E94D4316B017C0129A13AA14BA15CA1E4
:104EB00029966CAD7DAD8EAD9FAD29970E94D33103
:104EC0002D853E854F8558890E94A1349B01AC01F8
:104ED000C701B6010E94D4319B01AC010E94D431BC
:104EE0006B017C01A5019401C501B4010E94A134AC
:104EF0006D8B7E8B8F8B988FA5019401C501B401BA
:104F00000E94A1344B015C01A7019601C701B601C3
:104F10000E94A1349B01AC01C501B4010E94D431AF
:104F20000E9474354B015C012D8D3E8D4F8D58A133
:104F30006DA57EA58FA598A90E94D3316D8F7E8F18
:104F40008F8F98A329962CAD3DAD4EAD5FAD2997BF
:104F500069A17AA18BA19CA10E94D43169A37AA3F3
:104F60008BA39CA325962CAD3DAD4EAD5FAD259793
:104F700069A97AA98BA99CA90E94D3316D8B7E8BDC
:104F80008F8B988F2D8D3E8D4F8D58A16D817E8199
:104F90008F8198850E94A1346B017C0129A13AA1DF
:104FA0004BA15CA169857A858B859C850E94A13483
:104FB0009B01AC01C701B6010E94D4316B017C0199
:104FC0002D893E894F89588D6D857E858F8598897D
:104FD0000E94A1349B01AC01C701B6010E94D431EB
:104FE0009B01AC010E94D4316B017C0169962CAD10
:104FF0003DAD4EAD5FAD6997C301B2010E94A134D2
:1050000020E030E040E05FE30E94D3312DA13EA1DB
:105010004FA158A50E94D4316DA37EA38FA398A75A
:10502000A50194012D966CAD7DAD8EAD9FAD2D97F4
:105030000E94A1342B013C01A70196016D8D7E8D4C
:105040008F8D98A10E94A1349B01AC01C301B201D4
:105050000E94D43169A77AA78BA79CA7A5019401C8
:1050600061966CAD7DAD8EAD9FAD61970E94A13410
:105070002B013C01A701960169A17AA18BA19CA1FA
:105080000E94A1349B01AC01C301B2010E94D43142
:105090006DA77EA78FA798ABA501940165966CAD0F
:1050A0007DAD8EAD9FAD65970E94A1342B013C0173
:1050B000A70196016D897E898F89988D0E94A13400
:1050C0009B01AC01C301B2010E94D4316B017C0190
:1050D0002DA13EA14FA158A569AD7AAD8BAD9CAD78
:1050E0000E94A1344B015C0129A13AA14BA15CA112
:1050F00021966CAD7DAD8EAD9FAD21970E94A13400
:105100009B01AC01C501B4010E94D3314B015C018C
:10511000A701960169857A858B859C850E94A134BB
:105120002B013C012DA53EA54FA558A96D857E8577
:105130008F8598890E94A1349B01AC01C301B20103
:105140000E94D3319B01AC01C501B4010E94D4314E
:105150006D8B7E8B8F8B988F2D8D3E8D4F8D58A1B3
:1051600021966CAD7DAD8EAD9FAD21970E94A1348F
:105170004B015C012DA13EA14FA158A56DA97EA9AF
:105180008FA998AD0E94A1349B01AC01C501B40167
:105190000E94D3314B015C0129A53AA54BA55CA522
:1051A0006D857E858F8598890E94A1342B013C01F5
:1051B000A70196016D817E818F8198850E94A1341F
:1051C0009B01AC01C301B2010E94D3319B01AC0130
:1051D000C501B4010E94D4314B015C0129A13AA15F
:1051E0004BA15CA16DA97EA98FA998AD0E94A134A5
:1051F0006B017C012D8D3E8D4F8D58A169AD7AAD2F
:105200008BAD9CAD0E94A1349B01AC01C701B601DE
:105210000E94D3316B017C012DA53EA54FA558A955
:105220006D817E818F8198850E94A1342B013C0184
:1052300029A53AA54BA55CA569857A858B859C85B2
:105240000E94A1349B01AC01C301B2010E94D33181
:105250009B01AC01C701B6010E94D4316B017C01F6
:105260006091A8247091A9248091AA249091AB24E4
:1052700020E030E0A9010E94513418160CF0AAC0B9
:105280002091A8243091A9244091AA245091AB24C4
:10529000409098245090992460909A2470909B2478
:1052A0006D897E898F89988D0E94A1342AEF39EC0F
:1052B00044E359E30E94A134A30192010E94D43136
:1052C000609398247093992480939A2490939B24BC
:1052D0002091A8243091A9244091AA245091AB2474
:1052E0004090942450909524609096247090972438
:1052F000C501B4010E94A1342AEF39EC44E359E31B
:105300000E94A134A30192010E94D431609394249D
:105310007093952480939624909397242091A824A9
:105320003091A9244091AA245091AB24409090241C
:10533000509091246090922470909324C701B601FC
:105340000E94A1342AEF39EC44E359E30E94A134CE
:10535000A30192010E94D431609390247093912410
:1053600080939224909393242091982430919924AF
:1053700040919A2450919B2469897A898B899C89D0
:105380000E94D431698B7A8B8B8B9C8B20919424D7
:10539000309195244091962450919724698D7A8D6F
:1053A0008B8D9C8D0E94D431698F7A8F8B8F9C8FCF
:1053B00020919024309191244091922450919324F3
:1053C00069817A818B819C81EFD769837A838B8312
:1053D0009C8318C0109298241092992410929A24B9
:1053E00010929B241092942410929524109296244B
:1053F000109297241092902410929124109292244B
:105400001092932420910420309105204091062091
:10541000509107206D897E898F89988D0E94A134D3
:105420009B01AC0169897A898B899C89BDD7698B7D
:105430007A8B8B8B9C8B209104203091052040919E
:10544000062050910720C501B4010E94A1349B01A0
:10545000AC01698D7A8D8B8D9C8DA6D7698F7A8FE3
:105460008B8F9C8F20910420309105204091062045
:1054700050910720C701B6010E94A1349B01AC01E5
:1054800069817A818B819C818FD769837A838B83B1
:105490009C832AEF39EC44EB58E369897A898B893C
:1054A0009C890E94A1346D837E838F8398872AEF25
:1054B00039EC44EB58E3698D7A8D8B8D9C8D0E947D
:1054C000A13469877A878B879C872AEF39EC44EB74
:1054D00058E369817A818B819C810E94A1346D8718
:1054E0007E878F87988BE0900020F09001200091BC
:1054F000022010910320E98AFA8A0B8B1C8B809082
:10550000A4249090A524A090A624B090A724E09075
:10551000A024F090A1240091A2241091A324E98E4C
:10552000FA8E0B8F1C8F40909C2450909D2460908D
:105530009E2470909F24C0900020D0900120E09085
:105540000220F0900320C501B40190582D813E81C6
:105550004F8158850E94A13469837A838B839C8311
:10556000298D3A8D4B8D5C8D69857A858B859C85DF
:105570000E94A1349B01AC0169817A818B819C815D
:1055800012D769837A838B839C83A30192016D85F3
:105590007E858F8598890E94A1349B01AC01698129
:1055A0007A818B819C81FFD6A7019601FDD66093FD
:1055B000002070930120809302209093032040905C
:1055C0009C2450909D2460909E2470909F24C090B5
:1055D000A424D090A524E090A624F090A7242989A3
:1055E0003A894B895C896D817E818F8198850E9483
:1055F000A13469837A838B839C83298D3A8D4B8D6B
:105600005C8D6D857E858F8598890E94A1349B0174
:10561000AC0169817A818B819C81C6D669837A834A
:105620008B839C83A301920169857A858B859C85F8
:105630000E94A1349B01AC0169817A818B819C819C
:10564000B2D6A7019601B0D66093A4247093A52486
:105650008093A6249093A72440909C2450909D244E
:1056600060909E2470909F24C090A024D090A1248C
:10567000E090A224F090A32429893A894B895C897F
:1056800069857A858B859C850E94A13469837A839C
:105690008B839C83A50194016D857E858F85988978
:1056A0000E94A1349B01AC0169817A818B819C812C
:1056B0007AD669837A838B839C83A30192016D815F
:1056C0007E818F8198850E94A1349B01AC01698104
:1056D0007A818B819C8168D6A701960165D66093FB
:1056E000A0247093A1248093A2249093A324C0901B
:1056F0009C24D0909D24E0909E24F0909F242989A2
:105700003A894B895C896D857E858F8598890E9451
:10571000A1342B013C01A501940169857A858B8513
:105720009C850E94A1349B01AC01C301B2013CD60F
:105730004B015C01298D3A8D4B8D5C8D6D817E8195
:105740008F8198850E94A1349B01AC01C501B401F1
:105750002AD6A701960128D660939C2470939D2495
:1057600080939E2490939F2460910020709101204B
:1057700080910220909103202091002030910120FF
:1057800040910220509103208090A4249090A52461
:10579000A090A624B090A7244090A4245090A524C3
:1057A0006090A6247090A724E090A024F090A124FB
:1057B0000091A2241091A324ED82FE820F8318870A
:1057C000E090A024F090A1240091A2241091A324A1
:1057D000E986FA860B871C87E0909C24F0909D2434
:1057E00000919E2410919F24E982FA820B831C83EE
:1057F000E0909C24F0909D2400919E2410919F2481
:10580000ED86FE860F87188B0E94A1346B017C0108
:10581000A3019201C501B4010E94A1349B01AC0116
:10582000C701B601C1D54B015C0129853A854B857D
:105830005C856D817E818F8198850E94A1349B015A
:10584000AC01C501B401B0D54B015C012D853E858D
:105850004F85588969817A818B819C810E94A1340E
:105860009B01AC01C501B4019FD58B019C0135950D
:105870002795179507950F2EFFEDCF2EF9E5DF2E13
:10588000F7E3EF2EFFE5FF2EF02DC01AD10AE20A52
:10589000F30A20E030E040E05FE30E94A134A7017A
:1058A00096010E94A134A70196010E94A1349B0198
:1058B000AC0160E070E080EC9FE375D5A701960134
:1058C0000E94A1346B017C01609100207091012045
:1058D0008091022090910320A70196010E94A1349B
:1058E0006093002070930120809302209093032006
:1058F0006091A4247091A5248091A6249091A7245E
:10590000A70196010E94A1346093A4247093A5245A
:105910008093A6249093A7246091A0247091A12441
:105920008091A2249091A324A70196010E94A13402
:105930006093A0247093A1248093A2249093A32425
:1059400060919C2470919D2480919E2490919F242D
:10595000A7019601F6D760939C2470939D248093B1
:105960009E2490939F24C85ADF4FCDBFDEBFDF91A6
:10597000CF911F910F91FF90EF90DF90CF90BF904C
:10598000AF909F908F907F906F905F904F903F90DF
:105990002F90089581E08093AC240895FC018381C9
:1059A000A181B28194E0899FA00DB11D11241D92A7
:1059B0001D921D921C9213978381A181B28194E064
:1059C000899FA00DB11D11244D935D936D937C9320
:1059D00013972081838190E00196622F70E00E94EE
:1059E0001A3A83838481821710F48F5F8483089529
:1059F0004F925F926F927F928F929F92AF92BF92DF
:105A0000CF92DF92EF92FF920F931F93CF93DF938A
:105A1000FC01D481DD2309F47CC0B080DB1539F0B2
:105A2000B11053C080E0C12CD12C760163C001813C
:105A300012817801C0E0912C812CF70141905190A6
:105A4000619071907F01F80184E0989EE00DF11D56
:105A500011242081318142815381C301B20121D7B8
:105A600018168CF0F80184E0889EE00DF11D1124D9
:105A70002081318142815381C301B20172D58823D3
:105A80001CF48C2E01C09C2ECF5FDC13D6CFA12C32
:105A9000B12CC0E0C12CD12C76018C1671F09C1673
:105AA00061F0F801EA0DFB1D2081318142815381B3
:105AB000C701B60179D46B017C01CF5FE4E0AE0E83
:105AC000B11CDC13EACF82E015C001811281C0E075
:105AD000C12CD12C7601F801219131914191519144
:105AE0008F01C701B60160D46B017C01CF5FBC128E
:105AF000F2CF80E06D2F70E0681B7109072E000C5B
:105B0000880B990BCDD59B01AC01C701B6012DD5F2
:105B100003C060E070E0CB01DF91CF911F910F9146
:105B2000FF90EF90DF90CF90BF90AF909F908F90BD
:105B30007F906F905F904F900895FC011482408396
:105B4000618372830895FC018381A181B28194E015
:105B5000899FA00DB11D11241D921D921D921C92B2
:105B600013978381A181B28194E0899FA00DB11D1B
:105B700011244D935D936D937C93139720818381C2
:105B800090E00196622F70E00E941A3A838384812C
:105B9000821710F48F5F848308954F925F926F9203
:105BA0007F928F929F92AF92BF92CF92DF92EF92AD
:105BB000FF920F931F93CF93DF93FC01D481DD23DA
:105BC00009F47CC0B080DB1539F0B11053C080E01F
:105BD000C12CD12C760163C0018112817801C0E013
:105BE000912C812CF70141905190619071907F012F
:105BF000F80184E0989EE00DF11D1124208131818F
:105C000042815381C301B2014CD618168CF0F801C1
:105C100084E0889EE00DF11D1124208131814281B4
:105C20005381C301B2019DD488231CF48C2E01C082
:105C30009C2ECF5FDC13D6CFA12CB12CC0E0C12CA1
:105C4000D12C76018C1671F09C1661F0F801EA0DEA
:105C5000FB1D2081318142815381C701B601A4D34C
:105C60006B017C01CF5FE4E0AE0EB11CDC13EACF28
:105C700082E015C001811281C0E0C12CD12C7601D7
:105C8000F80121913191419151918F01C701B601E4
:105C90008BD36B017C01CF5FBC12F2CF80E06D2F04
:105CA00070E0681B7109072E000C880B990BF8D463
:105CB0009B01AC01C701B60158D403C060E070E09D
:105CC000CB01DF91CF911F910F91FF90EF90DF906B
:105CD000CF90BF90AF909F908F907F906F905F908C
:105CE0004F900895FC01148240836183728308956C
:105CF0001092AC2420E230E042E064E08DEA94E2CD
:105D00000E94E71264E68DEA94E20E94C113E091DA
:105D1000AD24F091AE2486818C7F8683868181605C
:105D200086836AEC7CE2CF010C947B0D089580E0C1
:105D30000C94291608958091AC2408951F920F9217
:105D40000FB60F92112408B60F9218BE2F933F93EF
:105D50004F935F936F937F938F939F93AF93209114
:105D6000A4293091A5294091A6295091A729609195
:105D7000A8297091A9298091AA299091AB29A1E025
:105D80000E94673A2093A4293093A5294093A6291D
:105D90005093A7296093A8297093A9298093AA29D1
:105DA0009093AB29AF919F918F917F916F915F916C
:105DB0004F913F912F910F9008BE0F900FBE0F9003
:105DC0001F9018958F929F92AF92BF92CF92DF92C1
:105DD000EF92FF920F931F93CF93DF93FC010190FB
:105DE0000020E9F731977F01E81AF90A47011E14EC
:105DF0001F040CF043C06C0110E0A12CB12C00E09A
:105E0000F601E10FF11DC0818C2F0C2E000C990BB7
:105E1000C0970A9738F0CD3221F581E0E81AF108F1
:105E200001E01FC081E0E81AF108B7010F2C000C57
:105E3000880B990B35D49B01AC0160E070E080E2E7
:105E400091E4E2D52DD60C2E000CDD0BE097F5D3B6
:105E5000C69F9001C79F300DD69F300D1124A20E12
:105E6000B31E1F5F812F90E0881599054CF2002327
:105E700041F0882799278A199B0904C080E090E0A7
:105E800001C0C501DF91CF911F910F91FF90EF905D
:105E9000DF90CF90BF90AF909F908F90089568E073
:105EA00070E280EB94E00E94210FE0EBF4E081814E
:105EB00088608183E4EFF4E281E0828781E090E012
:105EC000848395838087918784EB94E2868397838C
:105ED0000895E4EFF4E2808361834093B42481E089
:105EE00090E08087918740E0BF0180EB94E00C94C4
:105EF000360F08950F931F93CF93C42F8901E4EFBA
:105F0000F4E280836183842F90E08087918741E071
:105F1000BF0180EB94E00E94360FCC2381F0A4EB0C
:105F2000B4E2F801C1502C2F30E02F5F3F4F200F1B
:105F3000311F10828D918193E217F307D1F7CF9132
:105F40001F910F910895EF92FF920F931F93CF939C
:105F5000DF93CDB7DEB7DA95CDBFDEBFC65FDE4FCC
:105F6000E880F980CA50D140AE01425F5E4FC45F05
:105F7000DE4F68817981CC50D140CE0101960E94DC
:105F80009D3B6981662359F08E010E5F1F4FC7014B
:105F90000E949A0FF80161918F016111F8CFD3959A
:105FA000CDBFDEBFDF91CF911F910F91FF90EF909A
:105FB000089583EA9FE280933D2590933E2561E119
:105FC00070E280EA98E00E94BB10E0EAF8E083818A
:105FD0008063838308951F920F920FB60F9211244E
:105FE00008B60F9218BE09B60F9219BE0BB60F92E3
:105FF0001BBE2F933F934F935F936F937F938F932A
:106000009F93AF93BF93EF93FF9380EA98E00E9432
:10601000A20F8093AC298091AC29803611F40E94A4
:106020006512FF91EF91BF91AF919F918F917F91F9
:106030006F915F914F913F912F910F900BBE0F90F9
:1060400009BE0F9008BE0F900FBE0F901F901895BD
:10605000CF93DF93FC0120E030E0C62FD0E0DE01DB
:10606000022E02C0B595A7950A94E2F7A0FD508BC9
:106070002F5F3F4F31962830310589F740FF0AC026
:1060800041FF03C0FC01658302C0FC016683FC0183
:10609000618302C0FC016283DF91CF91089543E0E8
:1060A00050E068E080EC97E0D3DF40E058E164E046
:1060B00080EC97E0CDCF0895CF92DF92EF92FF92E0
:1060C0006B017C010E946C1EA70196016CD160934C
:1060D000A0297093A1298093A2299093A329FF90CE
:1060E000EF90DF90CF900895CF93DF9310923025FB
:1060F00080EE80933F2510923B2510923C25109214
:106100003D2510923E25CBDF0E94240288E00E94AC
:106110004312E0E4F6E080818860808384818860B7
:106120008483C0EAD6E08881886088838C81886017
:106130008C8360E486E00E94590260E183E00E9463
:10614000590260E283E00E94590260E186E00E9409
:10615000590262E081E00E94590261E083E00E94FE
:10616000590288E3888B898B24DF99DE0E94A41E64
:1061700087E08093A20078940E9457120E947714BF
:106180000E94AE150E94241C0E94C31C0E947A1E0D
:106190000E94EA14ADDDDF91CF910895A5DF0F2EA7
:1061A000F3E38F2EF0E29F2EF02D6894442443F801
:1061B0000F2EF0EA5F2EF02D0F2EF5E0CF2EF1E23C
:1061C000DF2EF02D0F2EF6E3EF2EF1E2FF2EF02D55
:1061D0000EE511E20F2EFFEF2F2EF0E23F2EF02DF5
:1061E0000F2EF3EB6F2EF1E27F2EF02DA895A3DD9D
:1061F00081119DDD0E94261681110E948A160E943F
:10620000B817882329F00E94D61A80E00E94B5179B
:106210000E94CB14882351F39F928F924F925F92EA
:10622000E0913D25F0913E25199561E08FEF94E2D4
:106230000E94F81561E08AE095E20E94D11D8CE190
:1062400095E20E94E61780E195E20E94C817CFEF21
:10625000D4E28C8D8F938B8D8F938A8D8F93898DC4
:106260008F93888D8F938F898F938E898F938D894C
:106270008F938C898F938B898F938A898F93898948
:106280008F93DF92CF924F925F92E0913D25F091F4
:106290003E25199588A58F938FA18F938EA18F93FB
:1062A0008DA18F938CA18F938BA18F938AA18F93B4
:1062B00089A18F9388A18F938F8D8F938E8D8F93CC
:1062C0008D8D8F93FF92EF924F925F92E0913D25DB
:1062D000F0913E2519952DB73EB72C5D3F4F2DBF50
:1062E0003EBF88858F938F818F938E818F938D8111
:1062F0008F938C818F938B818F938A818F938981E8
:106300008F931F930F934F925F92E0913D25F091F1
:106310003E2519958CE295E20E949114E0913D256D
:10632000F0913E258DB79EB70C968DBF9EBF88A974
:10633000811105C022E031E2822F932F02C0822D0D
:10634000932D9F938F93AFEFB4E29F968C919F977D
:106350001F928F939E968C919E971F928F939D96DE
:106360008C911F928F9385E891E29F938F934F9228
:106370005F921995A0903D25B0903E250E946C1E1D
:106380009F938F937F936F937F926F924F925F92C1
:10639000F50119950E9413142DB73EB72C5E3F4F9F
:1063A0002DBF3EBF23CF5058BB27AA270ED03FC2D8
:1063B00030D230F035D220F031F49F3F11F41EF48A
:1063C000EFC10EF4E095E7FBE5C1E92F41D280F380
:1063D000BA17620773078407950718F071F49EF5E2
:1063E00059C20EF4E0950B2EBA2FA02D0B01B90166
:1063F00090010C01CA01A0011124FF27591B99F03B
:10640000593F50F4503E68F11A16F040A22F232F46
:10641000342F4427585FF3CF469537952795A79596
:10642000F0405395C9F77EF41F16BA0B620B730B3D
:10643000840BBAF09150A1F0FF0FBB1F661F771FAE
:10644000881FC2F70EC0BA0F621F731F841F48F463
:10645000879577956795B795F7959E3F08F0B3CFE9
:106460009395880F08F09927EE0F979587950895D3
:106470009F939F77EEE389379E0720F4ECE0F2E0EC
:10648000B7D109C048D19058A2EA2AED3FE049ECC3
:106490005FE39BDFCCD10F9007FC90580895B9D1F2
:1064A00058F080E891E009F49EEFBAD128F040E876
:1064B00051E059F45EEF09C073C1ECC1E92FE078F7
:1064C000C7D168F3092E052AC1F3261737074807F5
:1064D000590738F00E2E07F8E02569F0E025E06452
:1064E0000AC0EF6307F8009407FADB01B9019D01C8
:1064F000DC01CA01AD01EF9347D099D10AD05F9179
:10650000552331F02BED3FE049E450FD49EC4CCFF1
:106510000895DF93DD27B92FBF7740E85FE31616B4
:10652000170648075B0710F4D92FBFD19F938F93AD
:106530007F936F9317D3E0E2F2E035D178D12F91BA
:106540003F914F915F9109D2DD2349F09058A2EA23
:106550002AED3FE049EC5FE3D0785D2736DFDF913D
:1065600066C1F4D008F481E008950CD060C158D120
:1065700040F04FD130F021F45F3F19F00BC15111C1
:106580008AC10EC165D198F39923C9F35523B1F39C
:10659000951B550BBB27AA2762177307840738F092
:1065A0009F5F5F4F220F331F441FAA1FA9F333D0F1
:1065B0000E2E3AF0E0E830D091505040E695001CA5
:1065C000CAF729D0FE2F27D0660F771F881FBB1F61
:1065D000261737074807AB07B0E809F0BB0B802D3B
:1065E000BF01FF2793585F4F2AF09E3F510568F087
:1065F000D1C051C15F3FECF3983EDCF386957795AF
:106600006795B795F7959F5FC9F7880F911D969588
:10661000879597F90895E1E0660F771F881FBB1FE4
:10662000621773078407BA0720F0621B730B840B91
:10663000BA0BEE1F88F7E095089504D06894B11165
:106640002AC108950DD188F09F5790F0B92F99274E
:10665000B751A0F0D1F0660F771F881F991F1AF06D
:10666000BA95C9F712C0B13081F014D1B1E00895E4
:1066700011C1672F782F8827B85F39F0B93FCCF365
:10668000869577956795B395D9F73EF49095809563
:10669000709561957F4F8F4F9F4F0895E89409C083
:1066A00097FB3EF490958095709561957F4F8F4F45
:1066B0009F4F9923A9F0F92F96E9BB279395F6955B
:1066C000879577956795B795F111F8CFFAF4BB0FD9
:1066D00011F460FF1BC06F5F7F4F8F4F9F4F16C03D
:1066E000882311F096E911C0772321F09EE8872FC7
:1066F000762F05C0662371F096E8862F70E060E083
:106700002AF09A95660F771F881FDAF7880F9695FB
:10671000879597F90895DF93CF931F930F938B017C
:10672000EC01EDE4F2E03FD082D09801AE018B01A4
:10673000EC0160E070E080E89FE335DED5D19801A0
:10674000AE010F911F91CF91DF9107C1990F000802
:10675000550FAA0BE0E8FEEF16161706E807F90733
:10676000C0F012161306E407F50798F0621B730BCE
:10677000840B950B39F40A2661F0232B242B252B4F
:1067800021F408950A2609F4A140A6958FEF811DF2
:10679000811D089597F99F6780E870E060E0089593
:1067A0009FEF80EC0895DF93CF931F930F93FF9299
:1067B000EF92DF927B018C01689405C0DA2EEF0125
:1067C000CCD0FE01E894A591259135914591559144
:1067D000AEF3EF01FADDFE019701A801DA9479F733
:1067E000DF90EF90FF900F911F91CF91DF9108956F
:1067F0009F938F937F936F93FF93EF939B01AC01D4
:10680000A0D0EF91FF91CFDF2F913F914F915F91FA
:1068100098C000240A94161617061806090608954B
:1068200000240A9412161306140605060895092E6C
:106830000394000C11F4882352F0BB0F40F4BF2BDB
:1068400011F460FF04C06F5F7F4F8F4F9F4F08951B
:1068500057FD9058440F551F59F05F3F71F0479511
:10686000880F97FB991F61F09F3F79F087950895F6
:10687000121613061406551FF2CF4695F1DF08C015
:10688000161617061806991FF1CF86957105610532
:1068900008940895E894BB2766277727CB0197F9DA
:1068A000089554DF08F48FEF08959B01AC0160E078
:1068B00070E080E89FE359CE0EF0A7C171CF6894D5
:1068C00069CFCEDFC8F39923D1F3C6F3DF93CF931B
:1068D0001F930F93FF92C92FDD2788232AF021975A
:1068E000660F771F881FDAF720E030E040E85FEBA3
:1068F0009FE3883920F0803E30F021968F7754DD79
:10690000E5E7F2E003C050DDE2EAF2E04CDF8B01A4
:10691000BE01EC01FB2E6F5771097595771F880B2F
:10692000990BBEDE28E132E741E35FE316D0AF2DDD
:106930009801AE01FF900F911F91CF91DF9145DD3E
:1069400076CF0BD074CF65DF28F06ADF18F095237F
:1069500009F020CF25CF11249ECF7ADFA0F3959F99
:10696000D1F3950F50E0551F629FF001729FBB2736
:10697000F00DB11D639FAA27F00DB11DAA1F649FE2
:106980006627B00DA11D661F829F2227B00DA11D95
:10699000621F739FB00DA11D621F839FA00D611D1B
:1069A000221F749F3327A00D611D231F849F600D3C
:1069B000211D822F762F6A2F11249F5750408AF075
:1069C000E1F088234AF0EE0FFF1FBB1F661F771F01
:1069D000881F91505040A9F79E3F510570F0DACEC4
:1069E0005ACF5F3FECF3983EDCF386957795679539
:1069F000B795F795E7959F5FC1F7FE2B880F911D1F
:106A00009695879597F90895FA01EE0FFF1F309636
:106A10002105310599F16115710561F48038BFE3F5
:106A20009B0749F168949038810561F08038BFEF89
:106A30009B0741F0992342F5FF3FE1053105210510
:106A400011F1E8940894E795D901AA2329F4AB2F12
:106A5000BE2FF85FD0F310C0FF5F70F4A695E0F78B
:106A6000F73950F019F0FF3A38F49F779F930CD024
:106A70000F9007FC905808953EF092CE60E070E0D1
:106A800080E89FE308954FE79F775F934F933F938D
:106A90002F9317DF2F913F914F915F9152DF6EC07F
:106AA000DFDEE0F09E37D8F09639B8F49E3848F42F
:106AB000672F782F8827985FF9CF86957795679508
:106AC00093959539D0F3B62FB1706B0F711D811D61
:106AD00020F487957795679593957CC096C0DBCE1B
:106AE00011F40EF45DCE91C0BBDED0F39923D9F33F
:106AF000CEF39F57550B87FF96D00024A0E640EABF
:106B0000900180585695979528F4805C660F771F02
:106B1000881F20F026173707480730F4621B730BD5
:106B2000840B202931294A2BA695179407942025F8
:106B300031254A2758F7660F771F881F20F0261740
:106B40003707480730F4620B730B840B200D311D9F
:106B5000411DA09581F7B901842F9158880F969512
:106B6000879508959B01AC01ECCEF0DD880B990B65
:106B7000089519F40EF00ECE8DCE12CE71DEC8F34C
:106B80009638C0F707F80F92E8942BE33AEA48EBFF
:106B90005FE7E5DE0F920F920F924DB75EB70F924F
:106BA0007FD0EFECF2E0FFDD4F915F91EF91FF912D
:106BB000E595EE1FFF1F49F0FE57E0684427EE0FF2
:106BC000441FFA95E1F74195550B36D00F9007FE1B
:106BD0006CCE0895882371F4772321F09850872B89
:106BE000762F07C0662311F499270DC09051862B8C
:106BF00070E060E02AF09A95660F771F881FDAF739
:106C0000880F9695879597F908959F3F31F0915099
:106C100020F4879577956795B795880F911D969580
:106C2000879597F9089591505040660F771F881FF8
:106C3000D2F70895AFCDE9CF13DEE8F39923D9F366
:106C4000940F511DBBF39150504094F059F088239C
:106C500032F0660F771F881F91505040C1F79E3F5A
:106C6000510544F7880F911D9695879597F90895DA
:106C70005F3FACF0983E9CF0BB2786957795679573
:106C8000B79508F4B1609395C1F7BB0F58F711F4AD
:106C900060FFE8CF6F5F7F4F8F4F9F4FE3CFFBCDFC
:106CA000FA01DC01AA0FBB1F9B01AC01BF5728F4FE
:106CB00022273327442750781FC0B75188F4AB2FC1
:106CC0000024469537952795011CA395D2F3002003
:106CD00069F0220F331F441FB395DAF30DD063CB55
:106CE00061307105A0E88A07B94630F49B01AC0118
:106CF0006627772788279078309621F02083318384
:106D00004283538308952F923F924F925F926F92E6
:106D10007F928F929F92AF92BF92CF92DF92EF922B
:106D2000FF920F931F93CF93DF93CDB7DEB760979A
:106D3000CDBFDEBF7C011B016A01FC0116821782F8
:106D4000838181FF2AC39E012F5F3F4F3901F701E5
:106D50009381F10193FD859193FF81911F01882318
:106D600009F417C3853239F493FD859193FF81911E
:106D70001F01853231F4B70190E0A3D456016501BB
:106D8000E6CF10E0512C912CFFE1F915D8F08B32B1
:106D900079F038F4803279F08332A1F4F92DF06182
:106DA0002EC08D3261F0803369F4292D21602DC011
:106DB000392D3260932E892D8460982E2AC0E92DBA
:106DC000E86015C097FC2DC020ED280F2A3088F40C
:106DD00096FE06C03AE0139F200D1124122F19C011
:106DE0008AE0589E200D1124522EE92DE0629E2E3D
:106DF00010C08E3231F496FCCCC2F92DF0649F2E77
:106E000008C08C3621F4292D2068922E02C08836C5
:106E100041F4F10193FD859193FF81911F0181114F
:106E2000B3CF9BEB980F933020F4992D9061805E47
:106E300007C09BE9980F933008F059C1992D9F7EA8
:106E400096FF16E09F73992E853619F49064992E5B
:106E500008C0863621F4392F3068932E02C01111F4
:106E6000115097FE07C01C3350F444244394410E44
:106E700027E00BC0183038F027E017E005C027E006
:106E80009CE3492E02C0212F412C560184E0A80E1C
:106E9000B11CF6016081718182819381042DA3016F
:106EA00022D36C01F981FC87F0FF02C0F3FF06C01A
:106EB00091FC06C092FE06C000E205C00DE203C0D0
:106EC0000BE201C000E08C858C7019F0011143C207
:106ED00080C297FE10C04C0CFC85F4FF04C08A8170
:106EE000813309F44A94141474F528E0241578F5D4
:106EF00088E0482E2CC096FC2AC0812F90E08C158B
:106F00009D059CF03CEFC3163FEFD30674F0892D2E
:106F10008068982E0AC0E2E0F0E0EC0FFD1FE10F60
:106F2000F11D8081803319F411501111F4CF97FEB7
:106F30000EC044244394410E812F90E0C816D90618
:106F40002CF41C1904C04424439401C010E097FEA3
:106F500006C01C141D0434F4C601019605C085E06A
:106F600090E002C081E090E001110196112331F020
:106F7000212F30E02F5F3F4F820F931F252D30E0F0
:106F80008217930714F4581A01C0512C892D897067
:106F900041F4552031F0B70180E290E092D35A9449
:106FA000F8CF002321F0B701802F90E08AD393FC23
:106FB00008C0552031F0B70180E390E082D35A94A5
:106FC000F8CF97FE4AC04601D7FE02C0812C912C13
:106FD000C60188199909F301E80FF91FED87FE87AB
:106FE0009601241931092F87388B012F10E0119554
:106FF000019511093FEF8316930621F4B7018EE244
:1070000090E05FD3C814D9044CF08F859889881517
:10701000990524F4ED85FE85818101C080E3F1E0CE
:107020008F1A91082D853E852F5F3F4F2D873E8714
:107030008016910624F0B70190E043D3DBCFC8144B
:10704000D90441F49A81963320F4953319F43C85A0
:1070500034FF81E3B70190E048C08A81813319F0A1
:107060009C859F7E9C87B70190E02BD3111105C0B2
:1070700094FC16C085E690E015C0B7018EE290E062
:1070800020D31E5F82E001E0080FF301E80FF11D3D
:107090008081B70190E015D3802F0113F4CFE8CFA2
:1070A00085E490E0B7010DD3D7FC06C0C114D1042C
:1070B00041F4EC85E4FF05C0D194C194D1088DE280
:1070C00001C08BE2B70190E0FCD280E32AE0C21657
:1070D000D1042CF08F5FFAE0CF1AD108F7CFB701B7
:1070E00090E0EFD2B701C601C096EBD249C183361A
:1070F00031F0833779F0833509F052C01FC0560153
:1071000032E0A30EB11CF6018081898301E010E01A
:10711000630111C05601F2E0AF0EB11CF601C08050
:10712000D18096FE03C0612F70E002C06FEF7FEF49
:10713000C601BCD28C01F92DFF7713C0560122E0A5
:10714000A20EB11CF601C080D18096FE03C0612F53
:1071500070E002C06FEF7FEFC6019DD28C01F92D68
:10716000F0689F2EF3FD18C0852D90E008171907D1
:1071700098F4B70180E290E0A4D25A94F5CFF601DA
:1071800097FC859197FE81916F01B70190E099D2AC
:1071900051105A94015011090115110581F7F0C0E1
:1071A000843611F0893659F5560197FE09C024E05E
:1071B000A20EB11CF60160817181828193810AC0A7
:1071C000F2E0AF0EB11CF60160817181072E000C58
:1071D000880B990BF92DFF769F2E97FF09C090958C
:1071E0008095709561957F4F8F4F9F4FF0689F2ED0
:1071F0002AE030E0A301C3D2C82EC6183EC0092D34
:10720000853721F40F7E2AE030E01DC0097F8F36DC
:1072100091F018F4883559F0BCC0803719F08837E0
:1072200011F0B7C0006104FF09C0046007C094FEFC
:1072300008C0066006C028E030E005C020E130E06C
:1072400002C020E132E0560107FF09C084E0A80E29
:10725000B11CF601608171818281938108C0F2E0E6
:10726000AF0EB11CF6016081718180E090E0A30156
:1072700086D2C82EC6180F77902E96FE0BC0092D09
:107280000E7FC11650F494FE0AC092FC08C0092D6E
:107290000E7E05C0DC2C092D03C0DC2C01C0D12ED4
:1072A00004FF0DC0FE01EC0DF11D8081803311F44F
:1072B000097E09C002FF06C0D394D39404C0802F76
:1072C000867809F0D39403FD10C000FF06C01C2D82
:1072D000D51478F4150D1D190CC0D51450F4B70150
:1072E00080E290E0EED1D394F8CFD51410F45D187D
:1072F00001C0512C04FF0FC0B70180E390E0E1D141
:1073000002FF16C001FD03C088E790E002C088E5D7
:1073100090E0B7010CC0802F867851F001FF02C0C9
:107320008BE201C080E207FD8DE2B70190E0C9D198
:10733000C11630F4B70180E390E0C3D11150F8CF0B
:10734000CA94F301EC0DF11D8081B70190E0B9D131
:10735000C110F6CF15C0F4E0F51550F584E0581AC9
:1073600093FE1EC0011125C02C8523FF27C008EF06
:1073700012E0392D3071932EF8018491811121C0D2
:10738000552009F4FCCCB70180E290E09AD15A94E0
:10739000F7CFF7018681978123C08FEF9FEF20C041
:1073A000B70180E290E08DD15A945110F9CFDACF35
:1073B000512CB701802F90E084D1D6CF0CEF12E092
:1073C000D8CF91108052B70190E07BD10F5F1F4F53
:1073D000D3CF23E0251510F483E0C1CF512CC4CFC7
:1073E0006096CDBFDEBFDF91CF911F910F91FF90CF
:1073F000EF90DF90CF90BF90AF909F908F907F9055
:107400006F905F904F903F902F900895AA1BBB1BE9
:1074100051E107C0AA1FBB1FA617B70710F0A61B94
:10742000B70B881F991F5A95A9F780959095BC01B5
:10743000CD01089597FB072E16F4009406D077FD32
:1074400008D0E4DF07FC05D03EF4909581959F4F6E
:107450000895709561957F4F0895A1E21A2EAA1B99
:10746000BB1BFD010DC0AA1FBB1FEE1FFF1FA217F4
:10747000B307E407F50720F0A21BB30BE40BF50BF1
:10748000661F771F881F991F1A9469F7609570957A
:10749000809590959B01AC01BD01CF010895EE0F41
:1074A000FF1F881F8BBF0790F691E02D1BBE19941C
:1074B000A29FB001B39FC001A39F700D811D112435
:1074C000911DB29F700D811D1124911D08950024FE
:1074D000A7FD00942A0F301D401D501D601D701D1A
:1074E000801D901D0895283008F027E03327DA0129
:1074F000990F311D87FD916000966105710539F482
:1075000032602E5F3D9330E32A95E1F708959F3F67
:1075100030F080387105610509F03C5F3C5F3D93B8
:10752000913008F08068911DDF93CF931F930F93E4
:10753000FF92EF92192F987F9695E92F9695969541
:10754000E90FFF27E65AFC4F99273327EE24FF2443
:10755000A701E70105900894079428F4360FE71E69
:10756000F81E491F511D660F771F881F991F06942B
:10757000A1F70590079428F4E70EF81E491F561F3F
:10758000C11D770F881F991F661F0694A1F70590EC
:10759000079428F4F80E491F561FC71FD11D880FE6
:1075A000991F661F771F0694A1F70590079420F492
:1075B000490F561FC71FD81F990F661F771F881FB7
:1075C0000694A9F784911095177041F0D695C79548
:1075D00057954795F794E7941A95C1F7E0E0F3E0E3
:1075E00068941590159135916591959105907FE27C
:1075F0007395E118F10A430B560BC90BD009C0F77C
:10760000E10CF11E431F561FC91FD01D7EF47033BD
:1076100011F48A95E6CFE894015030F0080F0AF48F
:107620000027021708F4202F2395022F7A3328F021
:1076300079E37D932A95E9F710C07D932A9589F621
:10764000069497956795379517951794E118F10A61
:10765000430B560BC90BD00998F023957E91739577
:107660007A3308F070E37C932013B8F77E91706151
:107670007D9330F0839571E37D9370E32A95E1F774
:107680001124EF90FF900F911F91CF91DF919927D7
:1076900087FD90950895FC010590615070400110A0
:1076A000D8F7809590958E0F9F1F0895FC0161502B
:1076B000704001900110D8F7809590958E0F9F1F14
:1076C00008950F931F93CF93DF93FB01238121FD37
:1076D00003C08FEF9FEF2CC022FF16C04681578159
:1076E000248135814217530744F4A081B1819D0163
:1076F0002F5F3F4F208331838C93268137812F5F0B
:107700003F4F2683378314C08B01EC01FB010084BB
:10771000F185E02D1995892BE1F6D80116968D910A
:107720009C911797019616968D939C931797CE016F
:10773000DF91CF911F910F9108950F931F93CF93D6
:10774000DF93CDB7DEB72E97CDBFDEBF8C0186E0CD
:107750008C8309831A838FEF9FE78D839E83CE01ED
:107760000196D1DAEF81F885E00FF11F10822E9695
:10777000CDBFDEBFDF91CF911F910F910895FA0128
:10778000AA27283051F1203181F1E8946F936E7F60
:107790006E5F7F4F8F4F9F4FAF4FB1E03ED0B4E051
:1077A0003CD0670F781F891F9A1FA11D680F791F92
:1077B0008A1F911DA11D6A0F711D811D911DA11DA3
:1077C00020D009F468943F912AE0269F11243019B3
:1077D000305D3193DEF6CF010895462F4770405D4E
:1077E0004193B3E00FD0C9F7F6CF462F4F70405DFD
:1077F0004A3318F0495D31FD4052419302D0A9F758
:10780000EACFB4E0A6959795879577956795BA9551
:10781000C9F700976105710508959B01AC010A2E17
:1078200006945795479537952795BA95C9F7620FEE
:0E783000731F841F951FA01D0895F894FFCFAD
:10783E000000803F0000C843801A060023000000AD
:10784E000000C201000300012D37383236002564D6
:10785E000A0024504D544B3235312C393630302AF3
:10786E0031370D0A00245047434D442C33332C300E
:10787E002A36440D0A0024504D544B3331342C30EB
:10788E002C312C302C302C302C302C302C302C3009
:10789E002C302C302C302C302C302C302C302C30FA
:1078AE002C302C302A32390D0A0024504D544B33D3
:1078BE0030302C3130302C302C302C302C302A32D1
:1078CE00460D0A0024504D544B3232302C35303098
:1078DE002A32460D0A0047524F554E4420414C5411
:1078EE003A20252D322E32660A00252D322E326692
:1078FE0009252D322E326609252D322E32660A00CA
:10790E004D505520494E495449414C495A45440A17
:10791E00004D414720464F554E440A00546573743E
:10792E002074656D703A20252D322E32660A005075
:10793E004D00414D00414343454C20583A20252DE2
:10794E00322E326609414343454C20593A20252DAB
:10795E00322E326609414343454C205A3A20252D9A
:10796E00322E32660A005941573A20252D322E32D8
:10797E00660950697463683A20252D322E326609E5
:10798E00526F6C6C3A20252D322E32660A00416CF5
:10799E007469747564653A20252D322E32660A4458
:1079AE0069676974616C2054656D703A20252D32BB
:1079BE002E32660A0054696D653A2048483A4D4D9C
:1079CE003A535320504D2F414D0A252D322E3264FD
:1079DE003A252D322E32643A252D322E3264202550
:1079EE00730A0054454D503A20252D322E32660A28
:0279FE00000087
:00000001FF
